:020000040000FA
:100000000C944F010C9477010C9477010C944225C9
:100010000C9442250C9442250C9477010C947701A2
:100020000C9477010C9477010C9477010C94770170
:100030000C9477010C9477010C9477010C94770160
:100040000C94F8240C9477010C94C6240C94A024EE
:100050000C9477010C9477010C9477010C94770140
:100060000C94BA250C94770107634236B79BD8A746
:100070001A39685618AEBAAB558C1D3CB7CC5763CD
:10008000BD6DEDFD753EF6177231BF000000803F7B
:1000900008000000BE922449123EABAAAA2ABECD97
:1000A000CCCC4C3E00000080BEABAAAAAA3E000009
:1000B0000000BF000000803F000000000008417801
:1000C000D3BB4387D1133D190E3CC3BD4282AD2B38
:1000D0003E68EC8276BED98FE1A93E4C80EFFFBE30
:1000E00001C4FF7F3F00000000004E414E494E49D1
:1000F0005459494E46CDCCCC3D0AD7233C17B7D1F5
:100100003877CC2B329595E6241FB14F0A0000209A
:10011000410000C84200401C4620BCBE4CCA1B0E19
:100120005AAEC59D7400407A10F35A00A0724E1862
:10013000090010A5D4E80000E87648170000E40B99
:1001400054020000CA9A3B000000E1F5050000805F
:10015000969800000040420F000000A086010000B9
:1001600000102700000000E8030000000064000009
:100170000000000A00000000000100000000002C48
:1001800076D888DC674F0823DFC1DFAE59E1B1B70D
:1001900096E5E3E453C63AE651997696E8E6C284DA
:1001A00026EB898C9B62ED407C6FFCEFBC9C9F40F2
:1001B000F2BAA56FA5F490055A2AF75C936B6CF917
:1001C000676DC11BFCE0E40D47FEF520E6B500D0ED
:1001D000ED902E0300943577050080841E08000002
:1001E000204E0A000000C80C333333330F986E12D0
:1001F000831141EF8D2114893BE65516CFFEE6DBD6
:1002000018D1844B381BF77C1D901DA4BBE424201F
:100210003284725E228100C9F124ECA1E53D270001
:100220005EBCE2613FDD83C29C7E20A3FD1F4100D6
:100230009D23BE46DB65F88C11AF32CA57E97400C6
:10024000000000240027002A00000000080002012E
:100250000000030407000000000000000000000090
:100260000023002600290000000000250028002BA4
:10027000000404040404040404020202020202034F
:100280000303030303010204081020408001020459
:1002900008102001020408102000D926052C112482
:1002A0001FBECFEFD8E0DEBFCDBF13E0A0E0B1E0CE
:1002B000ECECF1E702C005900D92A232B107D9F73C
:1002C00026E0A2E2B3E001C01D92A132B207E1F73D
:1002D00011E0CEE4D1E004C02197FE010E94563522
:1002E000CD34D107C9F70E9470280C94D9380C94EA
:1002F0000000089508950895AF92BF92CF92DF92C3
:10030000EF92FF920F931F93CF93DF936C017B01CA
:100310008B01040F151FEB015E01AE18BF08C0175B
:10032000D10759F06991D601ED91FC910190F081CE
:10033000E02DC6010995892B79F7C501DF91CF9191
:100340001F910F91FF90EF90DF90CF90BF90AF90F3
:100350000895CF93DF93FC014481558160817181C1
:100360008CE694E00E947C01EC0142E050E06BE5F9
:1003700071E08CE694E00E947C018C0F9D1FDF9160
:10038000CF910895FC01538D448D252F30E0842FAB
:1003900090E0821B930B541710F0CF9608950197AD
:1003A0000895FC01918D828D981761F0A28DAE0F9A
:1003B000BF2FB11D5D968C91928D9F5F9F73928F21
:1003C00090E008958FEF9FEF0895FC01918D828D4D
:1003D000981731F0828DE80FF11D858D90E008951A
:1003E0008FEF9FEF0895FC01918D228D892F90E072
:1003F000805C9F4F821B91098F73992708958CE62B
:1004000094E00E94F30121E0892B09F420E0822F7F
:10041000089580E090E0892B29F00E94FF0181116E
:100420000C9400000895FC01A48DA80FB92FB11DF4
:10043000A35ABF4F2C91848D90E001968F7399271A
:10044000848FA689B7892C93A089B1898C918370F8
:1004500080648C93938D848D981306C00288F389F1
:10046000E02D80818F7D80830895EF92FF920F931E
:100470001F93CF93DF93EC0181E0888F9B8D8C8D50
:1004800098131AC0E889F989808185FF15C09FB744
:10049000F894EE89FF896083E889F9898081837007
:1004A000806480839FBF81E090E0DF91CF911F91B6
:1004B0000F91FF90EF900895F62E0B8D10E00F5FD7
:1004C0001F4F0F731127E02E8C8D8E110CC00FB6AD
:1004D00007FCFACFE889F989808185FFF5CFCE0145
:1004E0000E941302F1CFEB8DEC0FFD2FF11DE35AAB
:1004F000FF4FF0829FB7F8940B8FEA89FB898081C8
:100500008062CFCFCF93DF93EC01888D8823B9F041
:10051000AA89BB89E889F9898C9185FD03C080810E
:1005200086FD0DC00FB607FCF7CF8C9185FFF2CF8B
:10053000808185FFEDCFCE010E941302E9CFDF91CC
:10054000CF910895833081F028F4813099F0823082
:10055000A9F008958730A9F08830C9F08430B1F44B
:10056000809180008F7D03C0809180008F77809381
:100570008000089584B58F7784BD089584B58F7DFC
:10058000FBCF8091B0008F778093B0000895809169
:10059000B0008F7DF9CFCF93DF93E8E5F2E084914F
:1005A000E4E9F2E0D491E0E8F2E0C491CC23A1F0D8
:1005B00081110E94A202EC2FF0E0EE0FFF1FE35A20
:1005C000FD4FA591B491EC91ED2381E090E009F409
:1005D00080E0DF91CF91089580E090E0FACF1F9303
:1005E000CF93DF93282F30E0F901E75BFD4F849133
:1005F000F901EB57FD4FD491F901EF58FD4FC4912C
:10060000CC23A9F0162F81110E94A202EC2FF0E05A
:10061000EE0FFF1FE959FD4FA591B4918FB7F894E4
:10062000EC91111108C0D095DE23DC938FBFDF91D0
:10063000CF911F910895DE2BF8CFCF93DF9390E0F9
:10064000FC01EB57FD4F24918F589D4FFC01849185
:100650008823D1F090E0880F991FFC01E15CFD4FE9
:10066000A591B491FC01E959FD4FC591D491611157
:100670000EC09FB7F8948C91E22FE0958E238C9357
:100680002881E223E8839FBFDF91CF9108958FB740
:10069000F894EC91E22BEC938FBFF6CF8E3008F0FC
:1006A0008E502091060190E4299F900111248770BB
:1006B000822B80937C0080917A00806480937A0002
:1006C00080917A0086FDFCCF80917800909179002E
:1006D00008953FB7F8948091E2039091E303A091CD
:1006E000E403B091E50326B5A89B05C02F3F19F0A0
:1006F0000196A11DB11D3FBFBA2FA92F982F8827A2
:10070000BC01CD01620F711D811D911D42E0660F7C
:10071000771F881F991F4A95D1F708958F929F924E
:10072000AF92BF92CF92DF92EF92FF926B017C016A
:100730000E9469034B015C01C114D104E104F1047E
:10074000B9F00E946903681979098A099B09683E12
:1007500073408105910580F321E0C21AD108E108B8
:10076000F10888EE880E83E0981EA11CB11CE4CF2E
:10077000FF90EF90DF90CF90BF90AF909F908F90C1
:1007800008958F929F92AF92BF92EF92FF921F9324
:10079000CF93DF93C82F1092150610921606109271
:1007A0001706109218061092190661E08FE00E9459
:1007B0001D0360E08FE00E94EF026C2F70E090E07C
:1007C00080E00E948E0360E08FE00E941D038BE9B1
:1007D00090E00197F1F7C0E9D1E00E94CB02892BAC
:1007E00071F42197D1F78EEF9FEFDF91CF911F9199
:1007F000FF90EF90BF90AF909F908F900895C0E9C9
:10080000D1E00E94CB02019719F42197D1F7EBCFE9
:10081000D8E2C0E810E090E9E92EFF24F3940E94AA
:10082000CB02892B29F481E0E81AF108C1F7DBCF6C
:100830000E9469034B015C0180E9E82EFF24F394D8
:100840000E94CB02019729F481E0E81AF108C1F770
:10085000CACF0E946903681979098A099B0969321C
:1008600071058105910538F0E12FF0E0E35FF94F64
:1008700080858C2B8087C69511F41F5FC0E8D1500E
:1008800051F690E080E0B1CF8F929F92AF92BF92ED
:10089000CF92DF92EF92FF920F931F93CF93DF934C
:1008A0008AE0A82EB12CD0E0C0E0EE24EA9493E0D8
:1008B000F92E88248A9423E0922ED12CC12C10E0AA
:1008C00000E08FE00E944E030817190790F1C81648
:1008D000D90608F46C018815990568F18E159F05F5
:1008E00008F47C01C80FD91F65E070E080E090E05B
:1008F0000E948E0381E0A81AB10819F70C0D1D1D86
:10090000CE01801B910B8E199F098819990966E009
:1009100070E00E942E35CB01DF91CF911F910F9196
:10092000FF90EF90DF90CF90BF90AF909F908F900F
:1009300008958C01D0CF4C01D5CF2FB7F89460919A
:10094000DE037091DF038091E0039091E1032FBFFC
:100950000895DC0180E0615090F09D919827E92F87
:10096000EF70F0E0E15EFD4F2491E92FE295EF702A
:10097000F0E0E15DFD4FE491822F8E27ECCF0895EA
:10098000DC012C911196ED91FC91F8948181822BE0
:1009900081839281322F30959323928387E090E078
:1009A0000197F1F781818323818383E290E00197AE
:1009B000F1F790817894EFECF0E03197F1F7922322
:1009C00081E009F480E00895FC0190810180F281CA
:1009D000E02D292F209560FF14C0F8948281822396
:1009E00082838181892B8183A3E2B0E01197F1F7A3
:1009F0008281982B9283789487ED90E00197F1F7AC
:100A00000895F8948281822382838181892B818356
:100A1000AFEFB0E01197F1F78281982B9283789431
:100A20008FE090E0EBCFDF92EF92FF920F931F9356
:100A3000CF93DF93EC01D62EE42E08E010E0FF24E4
:100A4000F39461E08D2D8F2109F460E0CE010E94C6
:100A5000E404FF0C01501109A1F7E11010C0F89453
:100A6000E981FA8191818881809589238183E98157
:100A7000FA81928188818095892382837894DF919D
:100A8000CF911F910F91FF90EF90DF900895EF921B
:100A9000FF920F931F93CF93DF938C017B0140E074
:100AA00065E50E941305E70188E0E80EF11C6991F5
:100AB00040E0C8010E941305CE15DF05C1F7DF91A4
:100AC000CF911F910F91FF90EF900895FC019081BD
:100AD0000180F281E02DF8948181292F20958223D5
:100AE000818378943DE743E050E0315029F1DA0109
:100AF0001197F1F780818923C1F3F89482818223D1
:100B000082838181892B81837894ABE7B7E0119749
:100B1000F1F7F894818182238183A3E1B1E01197F9
:100B2000F1F78081982381E009F080E07894E3E692
:100B3000F6E03197F1F7089580E008956F927F9283
:100B40008F929F92AF92BF92CF92DF92EF92FF92DD
:100B50000F931F93CF93DF93EC017B018A018E816A
:100B60009F810E946605811102C090E037C0B701E5
:100B70008E819F810E94470540E06EEB8E819F81B0
:100B80000E9413057801680189E0C80ED11CAE806F
:100B9000BF8088E0882E912C712C66246394C50157
:100BA0000E94C00481117628660CE1E08E1A91083B
:100BB000B1F7F70171927F01EC15FD0541F78E81C8
:100BC0009F810E946605813081F668E0C8010E941D
:100BD000A90491E0F80120852813C7CF892FDF9160
:100BE000CF911F910F91FF90EF90DF90CF90BF902A
:100BF000AF909F908F907F906F900895CF93DF93E9
:100C0000CDB7DEB729970FB6F894DEBF0FBECDBFC4
:100C1000AE014F5F5F4F0E949E05882331F08D81AA
:100C20008F33A9F020F48F31A1F080E007C08F3519
:100C300021F08F37D1F78CE001C08BE029960FB6F9
:100C4000F894DEBF0FBECDBFDF91CF9108958AE04B
:100C5000F5CF89E0F3CF2091F8033091F9032817FD
:100C6000390771F49091F6038091F703981741F0DA
:100C7000E091F603F0E0E356FC4F808190E00895A8
:100C80008FEF9FEF08950895EF92FF920F931F93B8
:100C9000CF93DF93DC015C96ED90FC905D97E114BF
:100CA000F10479F481E090E013969C938E9312976F
:100CB00090E080E0DF91CF911F910F91FF90EF9036
:100CC00008955196ED91FC91529750968C915097C2
:100CD000982F90950FB75E962C915E97122F1270F9
:100CE00021FD6095F8942081112319F1282B208390
:100CF000E7012197F1F728E0462F50E0308160FFAF
:100D00001AC0382B3083E7012197F1F7BA017595A6
:100D10006795215089F7112381F080818923808391
:100D20000FBF5C968D919C910197F1F781E090E067
:100D3000C1CF2923DCCF3923E5CF9081892BEFCF99
:100D40002091F8033091F9032817390771F4809145
:100D5000F7032091F60390E0805C9F4F821B91097E
:100D600060E470E00E944235089590E080E00895CC
:100D70002091F8033091F90328173907B9F49091BD
:100D8000F6038091F703981789F0E091F603F0E0FD
:100D9000E356FC4F80812091F60330E02F5F3F4FF8
:100DA0002F7333272093F60390E008958FEF9FEF82
:100DB00008950F931F930E949D046093F60570930E
:100DC000F7058093F8059093F9058EEE95E00E9463
:100DD000B80697FF1DC00E949D040091F605109172
:100DE000F7052091F8053091F905601B710B820B16
:100DF000930B0091F2051091F3052091F4053091C9
:100E0000F5056017710782079307F8F28FEF9FEFE0
:100E10001F910F910895E091F803F091F903E817FD
:100E2000F90769F4A389B4899C9185898095892300
:100E30008C931092F9031092F80381E0089580E0FA
:100E40000895109209061092080610920706109253
:100E5000060610920506109204068DE991E0909323
:100E60000B0680930A069091FA05963108F046C069
:100E70002DEB30E030930506209304062BE931E09A
:100E800030930706209306062CE231E030930906E2
:100E9000209308062091680084E0983048F031E003
:100EA0009E3008F430E081E001C0880F3A95EAF7FF
:100EB000822B809368002DE630E0983050F02BE6CE
:100EC00030E09E3030F02CE630E0963110F030E02B
:100ED00020E03093020620930106292F30E098305D
:100EE000C0F581E001C0880F9A95EAF78093030668
:100EF00080910A0690910B060197F1F78091080600
:100F000090910906892B21F18091F8039091F903C2
:100F100025E08E3E9207E1F0009711F00E940B074A
:100F200080910C068E7F80930C061092F70310922E
:100F3000F6038EEE95E09093F9038093F803E09129
:100F40000106F0910206808190910306892B80832F
:100F500008959E3040F42850310981E001C0880F87
:100F60002A95EAF7C3CF2E503109F7CF20917A03A3
:100F7000260F3327331F21323105ECF42091420430
:100F8000FC0190E080E0243069F082E00895A091B7
:100F90007A032191AC01465A5C4FA40FB52FB11DC5
:100FA0002C930196861798F380917A03680F6093CB
:100FB0007A0380E0089581E008951092420481E070
:100FC0008093410410921C0461E082E10E94EF02D0
:100FD00061E083E10E94EF02E9EBF0E080818E7F27
:100FE000808380818D7F808388E48093B80085E44E
:100FF0008093BC0008951092FB031092FA031092A4
:10100000490410926B040E94DD0789E791E09093F8
:10101000F5038093F4038AE791E09093F3038093C0
:10102000F2030895CF93DF9391E0909359038823BF
:10103000B9F0C091B800D091BA008091BC008A7B11
:101040008093BC0060E082E10E94EF0260E083E1F7
:101050000E94EF020E94DD07D093BA00C093B8004F
:10106000DF91CF910895CF92DF92EF92FF920F938D
:101070001F93CF93DF93D0916B0481E0D13208F0BE
:101080009CC0C0916A040E9469036B017C0180913D
:10109000420481116CC082E08093420481E080931D
:1010A00041048FEF8093400410923F04D0933E049C
:1010B000AAE4B4E0EEE1F4E080E0D8138DC0109231
:1010C0001D0480911D04CC0FC82BC0931D0480917A
:1010D0001C04813009F084C010921C040E94690332
:1010E0006B017C0180911D048093BB0080914404BE
:1010F00090914504A0914604B0914704892B8A2B16
:101100008B2BA1F00E9469030091440410914504C7
:1011100020914604309147046C197D098E099F097E
:10112000061717072807390708F442C08091BC004A
:1011300083FDD8CF85EC8093BC000E9469036B01CE
:101140007C0180914204823009F44CC080914004BB
:101150008F3F09F469C080914004803209F466C071
:1011600080914004803309F463C084E026C08091FC
:10117000440490914504A0914604B0914704892B02
:101180008A2B8B2B09F483CF0E94690300914404BE
:101190001091450420914604309147046C197D0953
:1011A0008E099F09061717072807390708F06FCF20
:1011B000809143040E94120885E010924904109225
:1011C0006B0410924804DF91CF911F910F91FF9013
:1011D000EF90DF90CF9008959D9191938F5F6DCFA9
:1011E00085EEA9CF8091440490914504A0914604D6
:1011F000B0914704892B8A2B8B2B09F4A2CF0E9434
:1012000069030091440410914504209146043091F3
:1012100047046C197D098E099F09061717072807CF
:10122000390708F08ECFC4CF80E0C7CF82E0C5CFAA
:1012300083E0C3CFCF92DF92EF92FF920F931F9381
:10124000CF93DF93D82FC62F613208F098C00E9449
:1012500069036B017C018091420481116BC081E0C4
:1012600080934204809341049FEF90934004109236
:101270003F049C0F90933E0480931D0480911D04B5
:10128000DD0FD82BD0931D0480911C04813009F010
:1012900078C010921C040E9469036B017C0180914C
:1012A0001D048093BB008091440490914504A0915B
:1012B0004604B0914704892B8A2B8B2BA1F00E9406
:1012C0006903009144041091450420914604309133
:1012D00047046C197D098E099F090617170728070F
:1012E000390708F448C08091BC0083FDD8CF85EC55
:1012F0008093BC000E9469036B017C0180914204D1
:10130000813009F440C080913F048C1710F4C091E3
:101310003F04EEE1F4E0ACEFB3E080E08C1355C0A5
:101320008C2FDF91CF911F910F91FF90EF90DF9065
:10133000CF9008958091440490914504A091460473
:10134000B0914704892B8A2B8B2B09F484CF0E9400
:1013500069030091440410914504209146043091A2
:1013600047046C197D098E099F090617170728077E
:10137000390708F070CF809143040E941208C0E042
:10138000CFCF85EEB5CF8091440490914504A091D4
:101390004604B0914704892B8A2B8B2B09F4AECFDE
:1013A0000E94690300914404109145042091460471
:1013B000309147046C197D098E099F09061717079C
:1013C0002807390708F09ACFD6CF91919D938F5F68
:1013D000A5CFE091FB038091FA03E81730F4F0E029
:1013E000E450FC4F808190E008958FEF9FEF0895C7
:1013F0009091FB038091FA032FEF3FEF981748F489
:10140000E92FF0E0E450FC4F208130E09F5F9093A3
:10141000FB03C90108958091FA039091FB03891B96
:10142000990B0895CF92DF92EF92FF920F931F9343
:10143000CF93DF937C01CB018A01209148042223C2
:1014400089F0EB016B01C40ED51ECC15DD0569F0EA
:101450006991D701ED91FC910190F081E02DC701D8
:101460000995F3CF642F0E94B607C801DF91CF9191
:101470001F910F91FF90EF90DF90CF900895CF9341
:10148000DF931F92CDB7DEB76983209148042223F2
:10149000F9F020916B04203258F021E030E0FC019B
:1014A0003383228390E080E00F90DF91CF91089505
:1014B00080914904E82FF0E0E65BFB4F998190832F
:1014C0008F5F8093490480936B0481E090E0ECCFC0
:1014D00061E0CE0101960E94B607F7CF90E080E070
:1014E00008958EEE95E00E940B070C9421072F9231
:1014F0003F924F925F926F927F928F929F92AF92A4
:10150000BF92CF92DF92EF92FF920F931F93CF93F0
:10151000DF93CDB7DEB72D970FB6F894DEBF0FBEC1
:10152000CDBF1C010E94710A64E670E080E090E08B
:101530000E948E036AE070E080E090E00E948E03DB
:10154000C101880F991F9D878C87D12CC12CF12C4C
:10155000E12C412C512C320149E050E06CE171E06A
:101560008EEE95E00E947C0165E070E080E090E006
:101570000E948E0310E000E0812C912C54018EEE2D
:1015800095E00E94A006892B39F4F4E08F169104AF
:10159000A104B1040CF05FC0023011050CF05BC077
:1015A0008EEE95E00E94A006892B99F08EEE95E0D4
:1015B0000E94B806E1E0F0E0EC0FFD1FE00FF11F24
:1015C00080836AE070E080E090E00E948E030F5F0D
:1015D0001F4F65E070E080E090E00E948E030230D3
:1015E000110509F070C089818F3F09F06CC08A81B4
:1015F000863809F068C0FE013396FB87EA878EEED5
:1016000095E00E94A006892B39F4F4E08F1691042E
:10161000A104B1040CF050C00930110509F059C003
:101620008B8190E0982F88272C81820F911D092EA5
:10163000000CAA0BBB0B480E591E6A1E7B1E40C035
:10164000EC85FD85EC15FD0509F086CFE114F1046C
:1016500041F4710106C08FEFC81AD80AE214F304EE
:101660007CF3C301B2010E9475304B015C01B701EC
:10167000FF0C880B990B0E9475309B01AC01C501D2
:10168000B4010E9493322D960FB6F894DEBF0FBEC0
:10169000CDBFDF91CF911F910F91FF90EF90DF9021
:1016A000CF90BF90AF909F908F907F906F905F9002
:1016B0004F903F902F900895043011050CF0B0CF5B
:1016C000FFEFEF1AFF0A8FEF881A980AA80AB80AE4
:1016D00056CF8EEE95E00E94B806EA85FB85819391
:1016E000FB87EA870F5F1F4F8ACF8F929F92AF923F
:1016F000BF92CF92DF92EF92FF92CF93DF93C0EC35
:10170000D5E0988121E02093480490936A041092D8
:10171000490410926B04682F89E095E00E943F0A0B
:101720000E94330863E088810E941A091092FB032B
:101730008093FA0389E095E00E94F809092E000CD5
:10174000AA0BBB0B8824982EA92EBA2E89E095E00F
:101750000E94F809092E000CAA0BBB0B6C017D013D
:10176000C828D928EA28FB28FE2CED2CDC2CCC2418
:1017700089E095E00E94F809BC01990F880B990B4C
:101780006C297D298E299F29DF91CF91FF90EF90C1
:10179000DF90CF90BF90AF909F908F9008958F92E1
:1017A0009F92AF92BF92CF92DF92EF92FF920F93F0
:1017B0001F932091C9052F3F19F48AEF0E94750BE2
:1017C0000091CD051091CE0530E020E0C72ED82E37
:1017D000E92EFF24E7FCFA94C01AD10AE20AF30AC0
:1017E00057E095958795779567955A95D1F7000FAE
:1017F000111F221F331F4B015C01801A910AA20A9C
:10180000B30AA5019401A091CF05B091D0050E9423
:10181000B6314B015C01FBE0B594A7949794879493
:10182000FA95D1F7A7019601C701B6010E941E35AE
:101830009B01AC01ACE05595479537952795AA9546
:10184000D1F7A091D105B091D2050E94B6319B018C
:10185000AC01BEE05595479537952795BA95D1F7D8
:10186000280D391D4A1D5B1D2093C5053093C60503
:101870004093C7055093C805A5E0B0E00E94AB3186
:1018800060587F4F8F4F9F4F672F782F892F992751
:1018900087FD9A950E94753020E030E048EC52E4D4
:1018A0000E9493321F910F91FF90EF90DF90CF90A5
:1018B000BF90AF909F908F9008952F923F924F923C
:1018C0005F926F927F928F929F92AF92BF92CF92D0
:1018D000DF92EF92FF920F931F93CF93DF93CDB7D9
:1018E000DEB76B970FB6F894DEBF0FBECDBF0E9478
:1018F000CF0B8091C9058F3F39F487EF0E94750B9C
:101900006E8B7F8B888F998F8091C5059091C605CE
:10191000A091C705B091C8056C017D01FF0CCC08F2
:10192000DC2C76019C01AD016C2D7C2D8C2D9C2D29
:10193000345F414051096109710981099109298781
:101940003A874B87652E762E872E982E9B8F5901CE
:10195000C42ED52EE62EF72E082F192F0E945C35A7
:10196000322E232E488B598B6A8B7B8B8C8B9D8BD5
:101970003091D6052091D505932F990F990B492FBA
:10198000592F692F792F892F0E945C350CE00E9416
:10199000543629833C874A8F5D876E877F87582E10
:1019A000492E3091D8052091D705932F990F990B87
:1019B000A32CB22CC888D988EA88FB880C891D8999
:1019C000492F592F692F792F892F0E945C3508E004
:1019D0000E946D36A980BC84CA8CDD84EE84FF84AD
:1019E000052D142D0E948A3670588F4F9F4FE0911D
:1019F000D305F091D4055F01D12CC12CE12CF12C41
:101A00008701E983BA82CB82DC82ED82FE820F837A
:101A10001887C12CD12CE12CF12C00E010E00E94A1
:101A20005C3501E20E946D362A8F532E49835C8714
:101A30006D877E878F87492EA0E00E949C3609F42F
:101A400036C13091DE052091DD05932F990F990B5A
:101A5000A32CB22CC888D988EA88FB880C891D89F8
:101A6000492F592F692F792F892F0E945C35190131
:101A7000488B598B6A8B7B8B8C8B9D8B3091DC05D3
:101A80002091DB05932F990F990BA984BA84CB84FD
:101A9000D62CE72CF82C092D1B8D492F592F692F97
:101AA000792F892F0E945C3501E10E945436510143
:101AB000C888D988EA88FB880C891D890E948A36E3
:101AC00059016A017B01382E192F4E895F89688D73
:101AD000798D84E075956795579547958A95D1F7E7
:101AE00080E090E0A0E1B0E0841B950BA60BB70B63
:101AF0003C014D01990C6608762C43019C01AD0117
:101B0000662D762D862D962D0FE10E945436722E6D
:101B1000832E942E5987B62FA72FF82FE92F3091B7
:101B2000DA052091D905932F990F990B492F592F39
:101B3000692F792F892F03E20E945436032D0E94CA
:101B40008A3659016A017B018C01272D382D492DD8
:101B500059856B2F7A2F8F2F9E2F0E949336E5E3A6
:101B6000AE2EFCE0BF2EC12CD12CE12CF12C00E0DC
:101B700010E00E945C35AA8CB52CC980DC84ED8411
:101B8000FE840F85142D0E94B6352F873E87498726
:101B90005A876B8779838C879D870DE00E946D360D
:101BA000922E832E742E652E562E472E382E292ED9
:101BB0003091E4052091E305932F990F990BA92CFF
:101BC000B82CC72CD62CE52CF42C032D122D492F24
:101BD000592F692F792F892F0E945C350E945C351F
:101BE00009E10E946D36AF84BE84C984DA84EB8437
:101BF000F9800C851D850E948A3619012A013B0156
:101C00004C013091E2052091E105932F990F990B3A
:101C1000492F592F692F792F892F0E945C3503E1B5
:101C20000E946D3659016A017B018C019101A2016C
:101C3000B301C4010E948A3608E00E946D36590142
:101C40006A017B01E82F192F3091E0052091DF0513
:101C5000932F990F990B492F592F692F792F892F7E
:101C600004E00E9454360E2F0E948A360E943B33B5
:101C700020E030E040E85BE30E94D4306B960FB682
:101C8000F894DEBF0FBECDBFDF91CF911F910F91B2
:101C9000FF90EF90DF90CF90BF90AF909F908F908C
:101CA0007F906F905F904F903F902F90089560E0ED
:101CB00070E0CB01E3CFBF92CF92DF92EF92FF9221
:101CC0000F931F93CF93DF93EC01B62EC72E8D8514
:101CD000811105C0CE010E94660581110EC01B86D0
:101CE0001D861C8680E0DF91CF911F910F91FF90A0
:101CF000EF90DF90CF90BF90089540E060EFCE016D
:101D00000E94130501E0E12CD12C11E0CE010E94CC
:101D1000C004F82ECE010E94C00491E0F91218C050
:101D2000813099F51134D8F2DB86D11002C081E000
:101D30008D878B81882399F22396EB2DFC2DCF0183
:101D4000089629912193E817F907D9F781E0CBCFBD
:101D5000EE2DF0E0F8120FC08B851817A0F4DE010D
:101D6000AE0FBF1F13968C91802379F4F12C19309C
:101D700008F41C87D12EEC0FFD1F8381902F9095C6
:101D8000892383830AC08113F1CFFE01EE0DF11D7B
:101D90008381802B8383FF24F3946F2DCE010E94D7
:101DA000E4041F5F000F11F4E39401E087E08E1557
:101DB00008F0ACCFB7CFDF92EF92FF920F931F9353
:101DC000CF93DF937C018B01D42EDC011696ED912D
:101DD000FC9113861586148612861186108617824A
:101DE0001682158214821382C0E0B801F701868141
:101DF00097810E945B0ED82F882329F0DC1629F0EA
:101E0000CF5FDC1690F7D0E009C067E0C8010E9400
:101E1000A904D80117969C918913F2CF8D2FDF91D9
:101E2000CF911F910F91FF90EF90DF900895CF9386
:101E30009091C9059F3F41F5682F8091C00591E0C1
:101E40009093480480936A041092490410926B04A2
:101E500089E095E00E943F0A0E94330862E0809189
:101E6000C0050E941A091092FB038093FA0389E0CF
:101E700095E00E94F809C82F89E095E00E94F809D2
:101E800020E03C2F282B392B922F832FCF910895C0
:101E90000F931F93CF93DF93FC01048115810115EC
:101EA000110539F4FB011082DF91CF911F910F9141
:101EB0000895415051094017510708F48A01EB0178
:101EC000FC0160817181A801CE010E94B038C00F71
:101ED000D11F1882E9CFCF93DF93C091B405D09181
:101EE000B505209761F08991882349F0082E000CF0
:101EF000990B0E948A38FE0131978083F4CFDF91DD
:101F0000CF91089585ED8093BC0080914404909119
:101F10004504A0914604B09147040796A11DB11D48
:101F200023E0B695A795979587952A95D1F72091A7
:101F3000BC0024FD03C01092420408954091440463
:101F4000509145046091460470914704452B462BFF
:101F5000472B69F30097A105B10541F025E32A95C8
:101F6000F1F700000197A109B109E1CF8091430485
:101F70000C941208FC0180819181009711F00C945F
:101F8000552C60E070E0CB010895FB014481558140
:101F9000FC01248135812417350778F080819181F7
:101FA000009759F0FB01608171816115710529F07D
:101FB0000E94A23821E0892B09F020E0822F0895A9
:101FC0000F931F93CF93DF938C01EB01FC01808172
:101FD00091810097E1F06881798161157105A9F01F
:101FE000428153812C813D814217530770F00E943A
:101FF0009B388C819D81F801958384831D821C828E
:10200000DF91CF911F910F9108950E9444378881ED
:102010009981F801918380838A819B819383828354
:102020008C819D8195838483198218821B821A82F8
:10203000E5CFCF93DF93EC0188819981009711F070
:102040000E944437198218821D821C821B821A82C8
:10205000DF91CF910895FC0180819181009711F06B
:102060000C94443708950F931F93CF93DF93EC01A3
:1020700088819981009759F02A813B81261737077B
:1020800030F081E0DF91CF911F910F9108958B0186
:102090006F5F7F4F0E94CD37009759F099838883F7
:1020A0001B830A832C813D81232B59F7FC0110826D
:1020B000E8CF80E0E7CFEF92FF920F931F93CF938B
:1020C000DF936115710541F480E0DF91CF911F919D
:1020D0000F91FF90EF90089541155105B1F07B01EC
:1020E000EC010C811D81040F151FB8010E943310F3
:1020F000882351F3288139818C819D81B701820F1A
:10210000931F0E949B381D830C8381E0DECFFC016E
:1021100044815581608171818AEB95E00C945B105C
:102120000F931F93CF93DF9300D0CDB7DEB78C0111
:1021300069831A8241E050E0BE016F5F7F4F0E94C9
:102140005B10811103C0C8010E941910C8010F90D3
:102150000F90DF91CF911F910F910895CF93DF934F
:10216000EC01FB0101900020E9F73197AF01461B1C
:10217000570B0E945B10811103C0CE010E94191001
:10218000CE01DF91CF910895CF93DF93EC01FB0156
:1021900044815581608171810E945B10811103C06F
:1021A000CE010E941910CE01DF91CF910895EF92D8
:1021B000FF920F931F93CF93DF93EC017B018A0172
:1021C000BA010E94331081110BC0CE010E94191078
:1021D000CE01DF91CF911F910F91FF90EF90089565
:1021E0001D830C83B701888199810E949B38F0CFB1
:1021F000FB0101900020E9F73197AF01461B570B17
:102200000C94D7100F931F93CF93DF93CDB7DEB706
:1022100062970FB6F894DEBF0FBECDBF8C01CB0125
:10222000F8011182108213821282158214824AE010
:10223000BE016F5F7F4F0E947C2CBE016F5F7F4F9E
:10224000C8010E94F81062960FB6F894DEBF0FBE68
:10225000CDBFDF91CF911F910F910895CF93DF9361
:10226000EC01FB018617970749F0608171816115C8
:10227000710541F0448155810E94D710CE01DF9154
:10228000CF9108950E941910F9CFFC01118210829C
:1022900013821282158214820C942E11FC01118279
:1022A00010821382128215821482FB010190002099
:1022B000E9F73197AF01461B570B0C94D710AF923B
:1022C000BF92CF92DF92EF92FF920F931F93CF9323
:1022D000DF936C015B017A0189012417350720F433
:1022E0008F2D7901042F182F6DE571E0C6010E9432
:1022F0004E11D5011496CD91DC91EC16FD06E0F45B
:102300000C171D0708F4E801D501ED91FC91119718
:10231000EC0FFD1F108110826D917C916E0D7F1D61
:10232000C60161157105A1F00E94F810F5018081C8
:102330009181C80FD91F1883C601DF91CF911F91DA
:102340000F91FF90EF90DF90CF90BF90AF900895E6
:102350000E941910EBCFCF93DF93EC01FB01248196
:1023600035810E945F11CE01DF91CF9108950F93C7
:102370001F93CF93DF93CDB7DEB72C970FB6F894AA
:10238000DEBF0FBECDBFFC012481358112161306BE
:1023900064F48C01253131059CF40E94A90164E1AB
:1023A00070E080E090E00E948E032C960FB6F894C7
:1023B000DEBF0FBECDBFDF91CF911F910F9108956A
:1023C0002FE030E050E040E0BC01CE0107960E94D3
:1023D0005F114B855C856F8178858CE694E00E9467
:1023E0007C0169E170E080E090E00E948E034FE0A4
:1023F00050E0B801CE0101960E94AB11BE016F5FA3
:102400007F4FCE0107960E94E00FCE0101960E94F9
:102410002B10CE0107960E94A90164E170E080E0D4
:1024200090E00E948E036DE571E0CE0107960E9458
:10243000F810CE0107960E942B10B7CFEF92FF92B3
:102440000F931F93CF93DF93CDB7DEB7A1970FB64E
:10245000F894DEBF0FBECDBF7C01CB01BA01F701FE
:1024600011821082138212821582148242E0420F7E
:102470008E010F5F1F4F0E94332C009789F0BC0123
:10248000C7010E94F810A1960FB6F894DEBF0FBEE8
:10249000CDBFDF91CF911F910F91FF90EF900895E5
:1024A000C7010E941910EFCFFF920F931F93CF9394
:1024B000DF93EC01F62E08811981C8010E94953145
:1024C000F81621F06F2DC8010E949D31CE01DF91D9
:1024D000CF911F910F91FF900895EF92FF920F936C
:1024E0001F93CF93DF9300D0CDB7DEB705E115E0A2
:1024F000855195407C01C701800F911F9A83898384
:10250000F80161918F01CE0101960E945412F5E00D
:1025100003361F0781F785E195E00F900F90DF915B
:10252000CF911F910F91FF90EF900895EF92FF923E
:102530000F931F93CF93DF9300D0CDB7DEB709E69B
:1025400015E0895695407C01C701800F911F9A8341
:102550008983F80161918F01CE0101960E94541286
:10256000F5E000391F0781F789E695E00F900F909D
:10257000DF91CF911F910F91FF90EF9008952F92CF
:102580003F924F925F926F927F928F929F92AF9203
:10259000BF92CF92DF92EF92FF920F931F93CF9350
:1025A000DF93CDB7DEB76E970FB6F894DEBF0FBEE0
:1025B000CDBF68EA75E084EB95E00E942E110E9481
:1025C0006B0F6EE571E0CE0101960E944E11BE01C7
:1025D0006F5F7F4F84EB95E00E94C50F182FCE01EF
:1025E00001960E942B10112329F0F0E0E0E00995FC
:1025F00081E092C062E671E0CE0101960E944E1128
:10260000BE016F5F7F4F84EB95E00E94C50F182FCE
:10261000CE0101960E942B10112351F166E671E064
:10262000CE0101960E944E1160E975E0CE0101963F
:102630000E94C410BC018AEB95E00E942E11CE01CD
:1026400001960E942B106AEB75E0CE0101960E9464
:102650004511CE0101960E94B711CE0101960E944C
:102660002B106DE571E08AEB95E00E94F810C0CF69
:1026700060E771E0CE0101960E944E11BE016F5FCE
:102680007F4F84EB95E00E94C50F182FCE01019675
:102690000E942B10112359F064E771E08AEB95E05A
:1026A0000E94F81086E995E00E948710CCCF62E87E
:1026B00071E0CE0101960E944E11BE016F5F7F4F07
:1026C00084EB95E00E94C50F182FCE0101960E9461
:1026D0002B101123D1F127E030E046E050E068EA0A
:1026E00075E0CE0101960E945F11BE016F5F7F4FC2
:1026F00082EA95E00E94E00FCE0101960E942B1025
:1027000082EA95E00E94BA0F672B19F41092E80351
:102710006FCF81E08093E8036E960FB6F894DEBF2A
:102720000FBECDBFDF91CF911F910F91FF90EF9022
:10273000DF90CF90BF90AF909F908F907F906F90E1
:102740005F904F903F902F90089569E871E0CE011F
:1027500001960E944E11BE016F5F7F4F84EB95E0A2
:102760000E94C50F182FCE0101960E942B10112335
:1027700009F4B8C0809157039091580318161906B0
:102780000CF036CF88EC90E0909305018093040123
:102790008CE694E00E9482021D861E861F86188A9F
:1027A000CC24C394D12C40EC242E43E0342E5E0183
:1027B000FDE0AF0EB11C2E0121E1420E511C57E588
:1027C000652E53E0752E80915703909158038C1518
:1027D0009D050CF40DCF8091040190910501813C81
:1027E000934024F0309205012092040100910401ED
:1027F00010910501750148018A189B08C4018E0DCE
:102800009F1D0E949531F70181937F01E415F50525
:10281000A9F7C8010496909305018093040123E36E
:10282000E22E23E0F22E0F521340C8018E0D9F1DA1
:102830000E949531F70181937F016E167F06A9F7FB
:102840004D855E856F85788923E0CE0107960E94CD
:102850001E12BE01695F7F4FCE0101960E94451195
:102860006DE871E0CE0101960E94AE10BC018AEBCA
:1028700095E00E942E11CE0101960E942B10CE01F0
:1028800007960E942B1063E373E0CE0101960E942D
:102890004E11CE0101960E948710CE0101960E9432
:1028A0002B106AEB75E0CE0101960E944511CE0116
:1028B00001960E94B711CE0101960E942B108091C3
:1028C0000401909105018496909305018093040181
:1028D00064E170E080E090E00E948E03FFEFCF1A89
:1028E000DF0A71CF60E971E0CE0101960E944E11BE
:1028F000BE016F5F7F4F84EB95E00E94C50F182FDC
:10290000CE0101960E942B101123F1F126E030E058
:1029100045E050E068EA75E0CE0101960E945F1143
:10292000BE016F5F7F4F82EA95E00E94E00FCE010B
:1029300001960E942B1082EA95E00E94BA0F672B45
:1029400019F41092320354CE81E08093320388EC64
:1029500090E0909305018093040110925803109227
:10296000570310922E0310922F03109230031092EF
:1029700031030E949D0460932A0370932B0380937C
:102980002C0390932D0334CE66E971E0CE010196BD
:102990000E944E11BE016F5F7F4F84EB95E00E9455
:1029A000C50F182FCE0101960E942B10112309F498
:1029B00076C08091AC059091AD05079708F418CECC
:1029C00046E050E068EA75E0CE0101960E94AB1146
:1029D000BE016F5F7F4F82EA95E00E94E00FCE015B
:1029E00001960E942B108091A2059091A305C12C05
:1029F000D12C7601009721F00E94512C6B017C01B3
:102A0000C0920C01D0920D01E0920E01F0920F01E4
:102A10006DE971E08AEB95E00E94F81022E0B701C1
:102A2000A601CE0107960E941E12BE01695F7F4F6C
:102A3000CE0101960E9445116AEB72E0CE0101962B
:102A40000E94AE100E948710CE0101960E942B10AA
:102A5000CE0107960E942B106AEB75E0CE0101961D
:102A60000E944511CE0101960E94B711CE01019638
:102A70000E942B100E949D0428EE33E040E050E0BD
:102A80000E94F531CA01B9010E9473306093ED03D1
:102A90007093EE038093EF039093F003A9CD68EA5F
:102AA00071E0CE0101960E944E11BE016F5F7F4F13
:102AB00084EB95E00E94C50F182FCE0101960E946D
:102AC0002B10112309F462C08091AC059091AD05E3
:102AD000079708F48DCD46E050E068EA75E0CE0136
:102AE00001960E94AB11BE016F5F7F4F82EA95E0B5
:102AF0000E94E00FCE0101960E942B108091A2054A
:102B00009091A305C12CD12C7601009721F00E9451
:102B1000512C6B017C01C0920001D0920101E09226
:102B20000201F09203016FEA71E08AEB95E00E94E6
:102B3000F81021E0B701A601CE0107960E941E12EF
:102B4000BE01695F7F4FCE0101960E9445116AEB7D
:102B500072E0CE0101960E94AE100E948710CE0155
:102B600001960E942B10CE0107960E942B106AEB53
:102B700075E0CE0101960E944511CE0101960E949A
:102B8000B711CE0101960E942B1032CD6AEB71E095
:102B9000CE0101960E944E11BE016F5F7F4F84EB04
:102BA00095E00E94C50F182FCE0101960E942B10B0
:102BB000112341F126E030E044E050E068EA75E09E
:102BC000CE0101960E945F11BE016F5F7F4F82EAC6
:102BD00095E00E94E00FCE0101960E942B1082EA40
:102BE00095E00E94BA0F70931605609315057093D7
:102BF00009016093080180910A0190910B010E94E4
:102C00006D12F6CC6FEB71E0CE0101960E944E1171
:102C1000BE016F5F7F4F84EB95E00E94C50F182FB8
:102C2000CE0101960E942B101123B1F143E050E038
:102C300068EA75E0CE0101960E94AB11BE016F5F9C
:102C40007F4F82EA95E00E94E00FCE0101960E943C
:102C50002B1062EA75E0CE0101960E94451160E0FA
:102C6000CE0101960E949010BC0186E995E00E9479
:102C70002E11CE0101960E942B1040919A05509181
:102C80009B054115510509F4B6CF67E175E086E96A
:102C900095E00E94480FAFCF66EC71E0CE0101963F
:102CA0000E944E11BE016F5F7F4F84EB95E00E9442
:102CB000C50F182FCE0101960E942B10112309F485
:102CC00082C08091AC059091AD05409708F0CEC2CE
:102CD00042E050E068EA75E0CE0101960E94AB1137
:102CE000BE016F5F7F4F82EA95E00E94E00FCE0148
:102CF00001960E942B108091A2059091A305009748
:102D0000F1F10E94512C20E030E048EC52E40E94A6
:102D1000D4300E940533609321057093220580937F
:102D200023059093240563EC71E08AEB95E00E9403
:102D3000F8106091210570912205809123059091F2
:102D400024058B019C0100591F45214031090134A4
:102D50001C4921053105B8F062EA75E0CE01019603
:102D60000E94451169EC71E0CE0101960E94AE10FF
:102D70000E948710CE0101960E942B1039CC60E092
:102D800070E0CB01C0CF0E94753020E030E048EC0D
:102D900052E40E949332AB01BC0122E0CE010196C5
:102DA0000E941E12CE0101960E948710CE0101964C
:102DB0000E942B1043E050E066ED71E08AEB95E055
:102DC0000E945B1018CF6AED71E0CE0101960E945F
:102DD0004E11BE016F5F7F4F84EB95E00E94C50FDF
:102DE000182FCE0101960E942B101123F1F025E03F
:102DF00030E044E050E068EA75E0CE0101960E94C0
:102E00005F11BE016F5F7F4F82EA95E00E94E00F85
:102E1000CE0101960E942B1082EA95E00E94BA0F23
:102E20007093620560936105E6CE6FED71E0CE01AF
:102E300001960E944E11BE016F5F7F4F84EB95E0BB
:102E40000E94C50F182FCE0101960E942B1011234E
:102E500009F45EC009E110E0C12CD12C760180E1BB
:102E60000E944E03BC01990F880B990B0E9475308C
:102E70009B01AC01C701B6010E9427326B017C01A6
:102E80006AE070E080E090E00E948E03015011093A
:102E900031F720E030E040EA50E4C701B6010E947B
:102EA000D43020E030EC4FE754E40E94933220E02D
:102EB00030E048EC51E40E94933260933D057093FA
:102EC0003E0580933F059093400580910A019091C3
:102ED0000B010E946D1263EE71E08AEB95E00E9497
:102EE000F81040913D0550913E0560913F0570916D
:102EF000400522E0CE0107960E941E12BE01695FC6
:102F00007F4FCE0101960E9445116BEE71E021CEFC
:102F10006EEE71E0CE0101960E944E11BE016F5F10
:102F20007F4F84EB95E00E94C50F182FCE010196CC
:102F30000E942B10112309F45BCB43E050E064EBBB
:102F400075E0CE0107960E94AB11BE01695F7F4F0D
:102F5000CE0101960E94451160E0CE0101960E94CB
:102F60009010BC0182EA95E00E942E11CE010196DC
:102F70000E942B10CE0107960E942B1062EA75E08A
:102F8000CE0149960E94451162EF71E0CE01019693
:102F90000E944E118D8D9E8D892BC9F1098D1A8D40
:102FA00069817A81C8010E94BF38009781F1FC01D4
:102FB000E01BF10B8F01CE0101960E942B106DE5F5
:102FC00071E0CE0143960E944E116DE571E0CE0195
:102FD0000D960E944E1110161106E4F464EF71E094
:102FE000CE0101960E944E11CE0101960E94B711AA
:102FF000CE0101960E942B10CE010D960E942B103F
:10300000CE0143960E942B10CE014996BCCD0FEF06
:103010001FEFD1CFBE01675E7F4FCE010D960E949C
:103020002E11D12CC12C8AEF682E77247A9496E049
:10303000592E89899A89009709F409C1F5E0CF16BC
:10304000D104C9F36EEC72E0CE0101960E944E11DC
:10305000BE016F5F7F4FCE010D960E94C50F182FE6
:10306000CE0101960E942B101111CAC001E010E0A0
:10307000980150E040E0BE01635F7F4FCE010796AC
:103080000E945F11BE01695F7F4FCE0101960E94D1
:10309000451160E0CE0101960E949010BC01CE0166
:1030A00043960E942E11CE0101960E942B10CE0154
:1030B00007960E942B10BE016D5E7F4FCE010796D2
:1030C0000E9445118B859C85029708F49CC06EEC8C
:1030D00072E0CE0101960E944E11BE016F5F7F4FDC
:1030E000CE0107960E94C50FF82ECE0101960E94D0
:1030F0002B10FF2009F487C022E030E041E050E0CF
:10310000BE01695F7F4FCE0101960E945F11CE0123
:1031100001960E94BA0F4B017B01CE0101960E94DD
:103120002B1097FE03C02CE1E20EF11CB3016E19C7
:103130007F095C9C70015D9CF00C1124F701E7593C
:10314000FA4F76876587CE0107960E942B10B7014C
:103150006E587A4F44E050E0CE0143960E94480FEB
:103160003FEFC31AD30A89899A890817190708F00B
:1031700067C0A801BE01635F7F4FCE0101960E9428
:10318000AB11BE016F5F7F4FCE0143960E94E00FEF
:10319000CE0101960E942B10BE016D5E7F4FCE01C5
:1031A0000D960E942E11AD84BE84A114B10409F4C1
:1031B00040CF09891A8975010115110509F439CF24
:1031C00047014FEF841A940AF7018081082E000C02
:1031D000990B0E943D30892BD9F4015011090A0D39
:1031E0001B1DF8018081082E000C990B0E943D30B8
:1031F000892B81F00E151F0568F001501109F1CFE0
:1032000002E010E035CFCE0107960E94BA0F91CFB1
:103210007401D6CF0F5F1F4FA8014E195F095A8B5B
:10322000498BAE14BF0420F4B701C5010E94923847
:10323000ED85FE8589899A89E80FF91F1082F9CEFC
:103240006DE571E0CE010D960E94F810F2CEC092AD
:103250006B05CC2041F081E0809369058EE190E020
:103260000E949612C9CE10926905F8CF80E054CA28
:103270002F923F924F925F926F927F928F929F9286
:10328000AF92BF92CF92DF92EF92FF920F931F9374
:10329000CF93DF93CDB7DEB7CD54D1090FB6F894F5
:1032A000DEBF0FBECDBF7C016DE571E08AEB95E01E
:1032B0000E94F810C7010596059768F08091F10308
:1032C000811109C02CEEE2162FEFF20624F0F092E5
:1032D000EC03E092EB03F7017A96E432F10510F08B
:1032E0000C946E24EA58F64E0C945635F9236E244D
:1032F000F4236E246E246E246E246E246E246E24B9
:103300006E242A1B2A1B2A1B9A19841D2A1B821E23
:10331000561F2A1B2A1B882097209A206E242A1BBE
:103320002A1BA82047223E23CF23EA232A1B2A1B3D
:103330002A1B2A1B60E08FE00E941D03E4E9F2E0F3
:10334000E491E8A3E0E8F2E0E491F0E0EE0FFF1F83
:10335000E35AFD4F859194919AA389A31BA61DA6BC
:103360001CA6CE01809698878F831D821E821982AB
:1033700089E08A8381E08B838C831C8A1B8A1AA64E
:1033800019A618A61FA21EA21DA21CA21BA201E024
:10339000BE01625D7F4F8F8198850E945B0E8823FE
:1033A00009F45CC067E0CE018E960E94A9049DA935
:1033B0008913EECF898181111DC08F8198850E946C
:1033C0006605BE01625D7F4F8F8198850E9447052B
:1033D00040E064EB8F8198850E9413058F8198856A
:1033E0000E94C004182F8F8198850E9466051111D4
:1033F00001C009831A818EA5803111F40C947624C2
:10340000BE01625D7F4FCE0101960E94FE058117CD
:1034100090F48A818A838D818F5F8D838EA5883217
:1034200031F0B0F4803119F0823209F0B1CF8E81E1
:103430008F5F8E83ADCF8EA5803111F48CE0EACF03
:10344000BE01625D7F4FCE0101960E94FE05E2CF74
:103450008B3369F3823409F09BCFE9CF8F81988554
:103460000E94660540E06CEC8F8198850E941305F0
:10347000498164E48F8198850E9413058B8188239C
:1034800079F1EA81E9504EEEC42E42E0D42EE330C9
:1034900038F4F0E0EE0FFF1FEA5EFE4FC080D180EF
:1034A0008C81882309F461C0898181115EC00E94EA
:1034B0009D044B015C010D2C000CEE08FF088F8170
:1034C00098850E94C004813059F00E949D046C19B7
:1034D0007D098E099F09681579058A059B0578F392
:1034E0008CE08A83F12CE12C0FE59FE7D92E2FE1A8
:1034F000C22E3FE3B32E8D818E151F0409F00CF40C
:1035000099C04E2DBE01695C7F4FCE0101960E948D
:10351000DB0E1A811D3080F11CE08FA9803181F112
:10352000BE01695C7F4FCE0101960E94FE058117A6
:1035300009F478C0AE01425D5F4FBE01695C7F4F08
:10354000CE0101960E949E05882309F46BC08FA9C5
:10355000803109F467C01B3009F468C01C3091F059
:103560001A3009F065C0BAAA0EC0B601DD0C880B8E
:10357000990B0E948E03B4CF193078F619E0CDCFA5
:103580008CE0D5CFDAAA8F8198850E946605BE01AE
:10359000695C7F4F8F8198850E94470540E06EE40B
:1035A0008F8198850E94130540E068A98F819885D6
:1035B0000E94130540E069A98F8198850E94130538
:1035C0008FA9803131F040E06AA98F8198850E94EF
:1035D00013058F8198850E946605BE01695C7F4F47
:1035E0008F8198850E944705498168E48F8198857D
:1035F0000E94130564E170E080E090E00E948E0379
:103600008981882331F06AE070E080E090E00E94D8
:103610008E038F8198850E9466058A81811708F440
:10362000812F8A833FEFE31AF30A65CF0AABABCF52
:10363000CAAAA9CF0E8110E0053011050CF0F3C025
:103640000115110509F0F1C063E675E08AEB95E01C
:103650000E942E118091BE059091BF05892B09F41F
:10366000C2C06AEB75E0CE0101960E944511CE0101
:1036700001960E94B711CE0101960E942B106AEBB1
:1036800075E0CE0180960E94451180913203882317
:1036900009F4A5C080915703909158038431910596
:1036A0000CF09DC00091040110910501013CF3E074
:1036B0001F070CF094C00196909358038093570312
:1036C0000E949D04C0902A03D0902B03E0902C030D
:1036D000F0902D036C197D098E099F090E947330AB
:1036E00020E030E04AE754E40E94933260932E03D6
:1036F00070932F038093300390933103083C11059E
:1037000034F488EC90E0909305018093040180915B
:103710000401909105010EE213E09C012E5233400A
:103720007901C701800F911F9A838983D8016D9118
:103730008D01CE0101960E945412B3E002331B07A3
:1037400081F7E0900401F0900501C7010496909381
:10375000050180930401BE01605E7F4FCE0101969A
:103760000E94451160E0CE0101960E949010BC01BC
:103770008AEB95E00E942E11CE0101960E942B103B
:103780004091BE055091BF054115510531F063E3ED
:1037900073E08AEB95E00E94480F87E5C82E83E02E
:1037A000D82E03E313E0F701EF52F3407F01C70186
:1037B000800F911F9A838983D8016D918D01CE016D
:1037C00001960E945412C016D10689F78091040117
:1037D0009091050184969093050180930401CE0198
:1037E00080960E942B1064E670E080E090E00E94DA
:1037F0008E03C35BDF4F0FB6F894DEBF0FBECDBFA5
:10380000DF91CF911F910F91FF90EF90DF90CF90BC
:10381000BF90AF909F908F907F906F905F904F90F0
:103820003F902F90089504E010E06DE571E08AEB81
:1038300095E00E94F81081E4882E85E0982EB12C46
:10384000A12C4A2DBE01695C7F4FCE0101960E94DA
:10385000DB0E81114EC0C12CD12CBEEFEB2EB2EC91
:10386000FB2EF40141905190619071904F01A301A2
:103870009201C301B2010E94E433811108C0A30187
:103880009201C701B6010E9427326B017C01FFEF54
:10389000AF1ABF0A20E030E04CEF52ECC701B6018E
:1038A0000E946E3087FF71C0B501CE01C7960E949D
:1038B00002116BE871E0CE018E960E944E11BE019E
:1038C000695C7F4FCE018E960E94C41060E871E063
:1038D0000E94AE1063E675E00E94C4100E9487103B
:1038E000CE018E960E942B10CE01C7960E942B10FF
:1038F000BDC0AE01425D5F4FBE01695C7F4FCE012E
:1039000001960E949E05882309F4A5CF6FA570E05B
:10391000762F6627770F770F770F2EA548E0249F25
:1039200090011124262B372B8FA98031D1F46DA95A
:1039300070E08CA9DB01A81BB109CD019695982FE9
:103940008827979587950E944235CB014097B9010A
:10395000F3E0660F771FFA95E1F760789C01260F78
:10396000371F2138B4EE3B070CF475CFB901330F84
:10397000880B990B0E94753020E030E040E05CE35A
:103980000E94D4306B017C016CCF0330110509F427
:103990009FC0B501CE01C7960E9402116BE871E08D
:1039A000CE018E960E944E11BE01695C7F4FCE0102
:1039B0008E960E94C410BC018CE995E00E942E11E5
:1039C000CE018E960E942B10CE01C7960E942B101E
:1039D00022E0B701A601CE01C7960E941E126CE933
:1039E00075E0CE018E960E94451164E672E0CE012C
:1039F0008E960E94AE10BE01695C7F4F0E94C4107B
:103A0000BC018CE995E00E942E11CE018E960E9499
:103A10002B10CE01C7960E942B106AEB75E0CE01E9
:103A20008E960E9445116CE975E0CE018E960E943B
:103A3000C410BC018AEB95E00E942E11CE018E9637
:103A40000E942B106AEB75E0CE018E960E94451104
:103A500060E2CE018E960E949010BC018AEB95E048
:103A60000E942E11CE018E960E942B100A151B0566
:103A700009F0E7CE03301105A9F46BE072E0CE0146
:103A80008E960E944E116AEB75E0CE018E960E94D2
:103A9000C410BC018AEB95E00E942E11CE018E96D7
:103AA0000E942B106AEB75E0CE018E960E944511A4
:103AB00065E172E0CE018E960E94AE10BC018AEBE9
:103AC00095E00E942E11CE018E960E942B10C2CD41
:103AD00022E0B701A601CE018E960E941E12BE0101
:103AE000625D7F4FCE01C7960E94451160E2CE0114
:103AF000C7960E9490100E948710CE01C7960E9420
:103B00002B10CE018E96F2CE60E080E10E941D0364
:103B10008091F1038111EBC02AE030E040E050E0F9
:103B20002E962CAF3DAF4EAF5FAF2E9768E272E09E
:103B30008AEB95E00E94F810312C212C28961FAEBC
:103B4000289729961FAE2997C12CD12C760102E324
:103B500010E0812C912C540180E10E944E03092E2B
:103B6000000CAA0BBB0B880E991EAA1EBB1E65E09B
:103B700070E080E090E00E948E030150110961F72F
:103B800040903D0550903E0560903F057090400587
:103B9000C501B4010E94753020E030E040EA50E4F5
:103BA0000E94D43020E030E040E85AE30E94D43054
:103BB00020E030E048E452E40E949332A3019201F5
:103BC0000E94263220E030E040E751E40E94D430E9
:103BD0004B015C01A30192016AE979E989E390E470
:103BE0000E9426329B01AC01C501B4010E949332B0
:103BF00020E030E0A9010E94273220E030E040E2DE
:103C000051E40E94D4305B018C019B01AC01632D17
:103C1000722D28968FAD289729969FAD29970E94DF
:103C20006E3087FF08C03A2C2B2C28960FAF2897B0
:103C300029961FAF29979FEFC91AD90AE90AF90AED
:103C40002E962CAD3DAD4EAD5FAD2E972C153D059E
:103C50004E055F050CF07BCF6EE170E080E090E0F8
:103C60000E948E036FE272E08AEB95E00E94F810EA
:103C700022E0432D522D28966FAD289729967FADCF
:103C80002997CE0101960E941E12BE016F5F7F4FE1
:103C9000CE0180960E9445116CE372E0CE018096C1
:103CA0000E94AE10BC0182EA95E00E942E11CE0166
:103CB00080960E942B10CE0101960E942B1063E487
:103CC00072E0CE0101960E944E1162EA75E0CE01CB
:103CD00001960E94C4106AEB75E00E94C410BC01FA
:103CE0008AEB95E00E942E11CE010196EECE83E084
:103CF00090E0A0E0B0E02E968CAF9DAFAEAFBFAF2E
:103D00002E9714CF68EC70E080E090E00E948E0364
:103D10000E94710A64E670E080E090E00E948E03E9
:103D200062E370E080E090E00E948E0349E050E0A2
:103D30006CE171E08EEE95E00E947C0162E370E040
:103D400080E090E00E948E0303E010E08EEE95E0AC
:103D50000E94A006892B61F149E050E06CE171E01E
:103D60008EEE95E00E947C0165E070E080E090E0DE
:103D70000E948E03F12CE12C8EEE95E00E94A006AD
:103D800032E0E316F104A4F48EEE95E00E94A00662
:103D9000892B39F08EEE95E00E94B8064FEFE41AB9
:103DA000F40A65E070E080E090E00E948E03E4CFCA
:103DB00062E370E080E090E00E948E030150110900
:103DC00029F68AE090E00E94770A6B017C0120E0EE
:103DD00030E0A9010E946E30181634F08AE090E0BD
:103DE0000E94770A6B017C010BE010E020E030E0DC
:103DF00042ED53E4C701B6010E946E30181684F0FC
:103E00000150110969F068EC70E080E090E00E94D8
:103E10008E0383E090E00E94770A6B017C01E6CF7D
:103E200020E030E0A901C701B6010E946E301816EB
:103E30000CF00ACC20E030E048EC52E4C701B601B7
:103E40000E946E3021E087FF20E0B701A601CE017D
:103E500001960E941E12BE016F5F7F4F8AEB95E0B4
:103E60000E94E00FCE0101960E942B106AEB75E0D4
:103E7000CE0101960E94451167E472E0CE010196E1
:103E80000E94AE10BC018AEB95E00E942E11CE017B
:103E900001960E942B106BE472E0CE0101960E9405
:103EA0004E116AEB75E0CE01019617CF0E949D047A
:103EB0004B015C018EEE95E00E940B0764E670E01A
:103EC00080E090E00E948E030E94210764E670E08B
:103ED00080E090E00E948E0328961FAE2897D12C98
:103EE000C12C312C212C2A961FAE1EAE2A977CEDB8
:103EF000472E75E0572E612C712CCE0180962796A7
:103F00009FAF8EAF27970E949D04681979098A098F
:103F10009B09683B7B408105910508F06AC08EEEE5
:103F200095E00E94A006892B09F450C04092F2054A
:103F30005092F3056092F4057092F5050E94D9063F
:103F400097FD44C082349105C9F78E010F5F1F4F62
:103F500078010E94D90697FF40C089818D34B1F560
:103F6000C8014D9630E020E0D8014D918D01240F1D
:103F7000311D8A179B07C1F72E5B3F4F8E8D90E056
:103F8000982F88274F8D840F911D28173907F1F43A
:103F90008C8190E0982F88272D81FC01E20FF11D84
:103FA0002A96FFAFEEAF2A972E80312C322C222496
:103FB0008F81280E311CC884D12CDC2CCC2489851F
:103FC000C80ED11CF1E02896FFAF289762E370E09D
:103FD00080E090E00E948E0396CFF70181937F01ED
:103FE00027962EAD3FAD27972E173F0709F0B1CF8B
:103FF000B4CF0E949D04681979098A099B09683B1E
:104000007B4081059105A8F428963FAD289733237E
:1040100009F477C062E370E080E090E00E948E03D4
:104020008EEE95E00E940B0762E370E080E090E086
:104030007BC028964FAD2897442309F462C0B6018F
:10404000CE0180960E940211B101CE018E960E948F
:1040500002112A966EAD7FAD2A97CE01CF960E94AF
:104060000211BE01615C7F4FCE01C7960E944511CF
:1040700061E472E0CE01C7960E94AE10BE01625D9F
:104080007F4F0E94C41061E472E00E94AE10BE0136
:10409000605E7F4F0E94C41060E572E00E94AE1027
:1040A000BC0182EA95E00E942E11CE01C7960E94C3
:1040B0002B10CE01CF960E942B10CE018E960E941F
:1040C0002B10CE0180960E942B1066E572E08AEBE1
:1040D00095E00E94F8106AEB75E0CE0180960E9490
:1040E000451162EA75E0CE0180960E94C410BC01C1
:1040F0008AEB95E00E942E11CE0180960E942B1033
:1041000089CF63E675E08AEB95E00E942E1182CF9D
:104110008091F103882321F08AEB95E00E94A901A8
:1041200068EC70E080E090E00E948E0393CA1092E9
:10413000F10390CA81E08093F1038093710580912F
:10414000EB039091EC039093EA038093E90382CA16
:1041500064E670E080E090E00E948E0380910801A8
:10416000909109010B9731F580911A06882309F087
:10417000F89482E10E94C1038C0180911A06882381
:1041800009F078940115110509F4D5C080E090EC90
:10419000A9E7B4EC80930D0690930E06A0930F064A
:1041A000B09310068093110690931206A093130605
:1041B000B09314068091080190910901469731F55A
:1041C00080911A06882309F0F89481E00E94C103C7
:1041D0008C0180911A06882309F078940115110545
:1041E00009F40AC180E090ECA9E7B4EC80930D06D5
:1041F00090930E06A0930F06B093100680931106BD
:1042000090931206A0931306B093140664E670E030
:1042100080E090E00E948E03012B09F01BCAC09041
:104220001106D0901206E0901306F0901406C0928A
:104230002603D0922703E0922803F092290380916D
:104240000D0690910E06A0910F06B0911006809376
:10425000220390932303A0932403B09325036DE5D9
:1042600071E0CE0180960E944E1121E0B701A601B7
:10427000CE0101960E941E12BE016F5F7F4FCE01DC
:1042800080960E94E00FCE0101960E942B1060ECF8
:1042900071E0CE0101960E944E11BE01605E7F4F1B
:1042A000CE0101960E94C41066E672E00E94AE1034
:1042B000BC018AEB95E00E942E11CE0101960E946E
:1042C0002B1040912203509123036091240370919D
:1042D000250321E0CE0101960E941E12BE016F5FF0
:1042E0007F4FCE0180960E94E00FCE0101960E9482
:1042F0002B106AE672E0CE0101960E944E11BE01BB
:10430000605E7F4FCE0101960E94C4106DE672E0A0
:104310000E94AE100E948710CE0101960E942B10C1
:1043200064E670E080E090E00E948E03CE0180960B
:104330000E942B108FC910911506E09016066E2D65
:1043400070E090E080E00E9475302DEC3CEC4CEC8D
:104350005DE30E94D4304B015C01612F70E090E07E
:1043600080E00E9475309B01AC01C501B4010E9440
:10437000273260930D0670930E0680930F0690937C
:10438000100600911706F0901806602F6F7770E006
:1043900090E080E00E9475304B015C016F2D70E071
:1043A00090E080E00E9475302DEC3CEC4CEC5DE33D
:1043B0000E94D4309B01AC01C501B4010E94273298
:1043C00007FD18C0609311067093120680931306C0
:1043D00090931406812F8E0D800F8F0D01E010E059
:1043E00090911906891302C010E000E01195019523
:1043F0001109E0CE9058E6CF1091160600911506EF
:10440000609115067091160676276727762790E04B
:1044100080E00E9473302DEC3CEC4CEC5DE30E949C
:10442000D43060930D0670930E0680930F06909320
:104430001006E0901806F09017066F2D6F77762F14
:104440006E2D90E080E00E9473302DEC3CEC4CEC43
:104450005DE30E94D430F7FC18C06093110670939E
:1044600012068093130690931406812F800F8E0DF1
:104470008F0D01E010E090911906891302C010E041
:1044800000E0119501951109C1CE9058E6CF8091B9
:104490000701882309F4DEC80E945D0C2B013C0152
:1044A0000E94CF0B4B015C016091210570912205A8
:1044B00080912305909124050E94753020E030E022
:1044C00048EC52E40E9493326B017C010E945D0C27
:1044D00020E030E048EC52E40E949332A7019601BC
:1044E0000E94933221E03EED42E45EE30E94943369
:1044F0006B017C0120E030E048EC52E4C301B201E2
:104500000E949332AB01BC0122E0CE0180960E9452
:104510001E12BE01605E7F4FCE0101960E944511C2
:104520006FE672E0CE0101960E94AE10BC018CE9EC
:1045300095E00E942E11CE0101960E942B10CE0113
:1045400080960E942B106CE975E082EA95E00E944B
:104550002E1166EC71E0CE0101960E944E116CE9BD
:1045600075E0CE0101960E94C410BC018CE995E073
:104570000E942E11CE0101960E942B1021E0B50160
:10458000A401CE0180960E941E12BE01605E7F4F84
:10459000CE0101960E94451164E772E0CE010196BA
:1045A0000E94AE10BC018AEB95E00E942E11CE0154
:1045B00001960E942B10CE0180960E942B1060EC79
:1045C00071E0CE0101960E944E116AEB75E0CE01BA
:1045D00001960E94C41067E772E00E94AE10BC0111
:1045E0008AEB95E00E942E11CE0101960E942B10BD
:1045F000A701960160E070E080E89FE30E94263208
:1046000020E03AE24DE257E40E94D430AB01BC0115
:1046100021E0CE0180960E941E12BE01605E7F4F97
:10462000CE0101960E94451169E472E0CE01019627
:104630000E94AE100E948710CE0101960E942B109E
:10464000CE0180960E942B106CE975E0CE01019698
:104650000E9445116AEB75E0CE0101960E94C410DC
:10466000BC018AEB95E00E942E11CE0101960E94BA
:104670002B1065E070E080E090E056CD9BE0E92EE5
:10468000F12C10E000E09924939423E2822E909282
:10469000480480926A041092490410926B0462E00C
:1046A00083E20E941A091092FB038093FA0389E0C7
:1046B00095E00E94F809D82EC12C89E095E00E946F
:1046C000F8095C01AC28BD280E943308B50190E0D0
:1046D00080E00E9473302AE939E949E95FE30E94EA
:1046E00093320E940C330617170708F48B0162E31C
:1046F00070E080E090E00E948E0351E0E51AF1083E
:1047000031F66BE772E08AEB95E00E94F81019A28F
:1047100018A21BA21AA21DA21CA24AE0BE016F5F32
:104720007F4FC8010E949C2CBE016F5F7F4FCE015E
:1047300080960E94F810BE01605E7F4FCE01019608
:104740000E9445116BE872E0CE0101960E94AE1006
:10475000BC0182EA95E00E942E11CE0101960E94D2
:104760002B10CE0180960E942B1060E972E0CE01E2
:1047700001960E944E1162EA75E0CE0101960E94F8
:10478000C4106AEB75E00E94C410BC018AEB95E08E
:104790000E942E11CE0101960E942B1045CC81E083
:1047A000809306010E9444048C0163E972E08AEB65
:1047B00095E00E94F81060E074E0601B710BCE0180
:1047C00001960E940211CE0101960E948710CE012F
:1047D0000196AECD63EA72E08AEB95E00E94F81094
:1047E0000E944404BC01EBCFF0E0E0E009950C949A
:1047F0002A1B80916B0518160CF057C081E080933E
:1048000069056EEA72E08AEB95E00E94F8108091EB
:104810006905882309F44CC06CEB72E0CE01019667
:104820000E944E116AEB75E0CE0101960E94C41001
:10483000BC018AEB95E00E942E11CE0101960E94E8
:104840002B106AEB75E0CE0101960E944511CE0156
:1048500001960E94B711CE0101960E942B1068EEBE
:1048600073E080E090E00E948E03809169058111E1
:104870000E947C246DE571E08AEB95E00E94F810BF
:104880008091F1038093710581110C942A1B6DECCA
:1048900072E08EEA95E00E94F81086EE9FEF90930A
:1048A000EC038093EB030C942A1B10926905A9CFAB
:1048B00064EC72E0CE0101960E944E116AEB75E045
:1048C000CE0101960E94C410BC018AEB95E00E94C3
:1048D0002E11CE0101960E942B10D2CF60ED72E016
:1048E0008AEB95E00E94F8100C942A1B1D3010F002
:1048F0000C94091A0C941E1A0F931F93CF93DF93F5
:1049000009E615E0D0E0C0E00A5F1F4F80916B051B
:10491000082E000C990BC817D9076CF4F801878191
:1049200090850E94381968EE73E080E090E00E9464
:104930008E032196E9CFDF91CF911F910F910895BA
:104940001F920F920FB60F9211242F933F934F9304
:104950005F936F937F938F939F93AF93BF93EF93E7
:10496000FF938CE694E00E941302FF91EF91BF91B8
:10497000AF919F918F917F916F915F914F913F91F7
:104980002F910F900FBE0F901F9018951F920F92AE
:104990000FB60F9211242F938F939F93EF93FF9352
:1049A000E0917C04F0917D048081E0918204F0919B
:1049B000830482FD1BC09081809185048F5F8F737B
:1049C00020918604821741F0E0918504F0E0E459DB
:1049D000FB4F958F80938504FF91EF919F918F916D
:1049E0002F910F900FBE0F901F9018958081F4CFDC
:1049F0001F920F920FB60F9211242F933F938F9314
:104A00009F93AF93BF938091DE039091DF03A091BA
:104A1000E003B091E1033091DD0323E0230F2D3754
:104A200058F50196A11DB11D2093DD038093DE038F
:104A30009093DF03A093E003B093E1038091E2033E
:104A40009091E303A091E403B091E5030196A11DC9
:104A5000B11D8093E2039093E303A093E403B0932A
:104A6000E503BF91AF919F918F913F912F910F904F
:104A70000FBE0F901F90189526E8230F0296A11DD8
:104A8000B11DD2CF1F920F920FB60F9211242F9308
:104A90003F934F935F936F937F938F939F93AF93C6
:104AA000BF93EF93FF93E091F803F091F9033097F0
:104AB00049F0A685B7858585968D91FF14C09C9198
:104AC0008923A1F4FF91EF91BF91AF919F918F91B5
:104AD0007F916F915F914F913F912F910F900FBEFA
:104AE0000F901F9018959C91892361F7A389B48931
:104AF0009C918589809589238C93868997890197D4
:104B0000F1F7608D718DA685B785558538E020E079
:104B1000CB010197F1F7822F90E095958795282F8B
:104B20004C91452309F02068315091F7868D81FD25
:104B300020958091F70390E001968F73992730912B
:104B4000F603381799F0A091F703B0E0A356BC4FD5
:104B50002C938093F703828D938D0197F1F7A389AE
:104B6000B4898C919589892B8C93ACCF868D81608B
:104B7000868FF1CF1F920F920FB60F9211242F93B1
:104B80003F934F935F936F937F938F939F93AF93D5
:104B9000BF93EF93FF938091B900887F803609F42B
:104BA0004AC0F0F5883209F4A7C018F5803109F43D
:104BB0009BC0B8F4882309F4F9C0883009F494C084
:104BC000FF91EF91BF91AF919F918F917F916F91E5
:104BD0005F914F913F912F910F900FBE0F901F90BB
:104BE0001895883109F488C0803251F780934004C9
:104BF00014C0803409F49DC040F48033B9F3883385
:104C0000F9F68093400485ECB0C0803509F485C086
:104C1000883509F496C0883499F60E94820FD0CF67
:104C2000883909F48CC038F5883729F050F4883673
:104C300011F0803729F683E08093420410929C03A0
:104C400057C0883809F47BC0803919F0803809F0E2
:104C5000B7CF80919C03803208F071C0E0919C0333
:104C600081E08E0F80939C038091BB00F0E0E458BC
:104C7000FC4F80833DC0803B39F0E0F4803A09F47A
:104C800079C0883A09F09CCF84E080934204109266
:104C90007B0310927A03E091F403F091F5030995F8
:104CA00080917A0381110FC081E080937A03109282
:104CB0005A0309C0803C09F4A6CF883C09F4A3CF6D
:104CC000883B09F07DCFE0917B0381E08E0F8093DC
:104CD0007B03F0E0E65AFC4F80818093BB0090910B
:104CE0007B0380917A0329C080911D048093BB00CF
:104CF00085EC8093BC0064CF90913F0480913E048A
:104D0000981758F5E0913F0481E08E0F80933F049F
:104D1000F0E0E25EFB4F8081E9CFE0913F0481E06B
:104D20008E0F80933F048091BB00F0E0E25EFB4F6A
:104D3000808390913F0480913E049817C8F285E8E3
:104D4000D8CFE0913F0481E08E0F80933F048091A3
:104D5000BB00F0E0E25EFB4F808380914104811153
:104D60005CCF81E080931C0484EA8093BC001092A5
:104D7000420426CF85EC8093BC00109242048091BF
:104D80009C03803230F4E0919C03F0E0E458FC4F47
:104D9000108260919C0370E0E091F203F091F303C4
:104DA0008CE793E0099510929C030ACF109240047F
:104DB00034CF10926F0410926E0488EE93E0A0E05E
:104DC000B0E08093700490937104A0937204B09348
:104DD000730429E231E030936D0420936C0425ECD8
:104DE00030E0309379042093780424EC30E0309361
:104DF0007B0420937A0420EC30E030937D042093F0
:104E00007C0421EC30E030937F0420937E0422EC7C
:104E100030E0309381042093800426EC30E030931E
:104E200083042093820410928504109286041092C9
:104E300087041092880410920C0510920B05809341
:104E40000D0590930E05A0930F05B09310052BE36D
:104E500031E030930A052093090510921A0610924A
:104E6000F1051092F0058093F2059093F305A0935D
:104E7000F405B093F5058DE491E09093EF058093F0
:104E8000EE05109205061092040610920706109285
:104E90000606109209061092080610920B06109250
:104EA0000A0660910C066E7F6D7F60930C06669516
:104EB000617081E0682789E00E94EF0261E089E08B
:104EC0000E941D03EEE8F2E0E491E093FE05EAE7BC
:104ED000F2E0E491F0E0EE0FFF1FE959FD4F8591FC
:104EE0009491909300068093FF0560E08AE00E9411
:104EF0001D0380910C0681FD04C061E08AE00E94E0
:104F0000EF028AE08093FA05EFE8F2E0E491E093A3
:104F1000FB05EBE7F2E0E491F0E0EE0FFF1FE35A50
:104F2000FD4F859194919093FD058093FC058FEF43
:104F30008093C9058093CA058093CB058093CC05E7
:104F40006DE571E08AEB95E00E944E116DE571E030
:104F500084EB95E00E944E116DE571E08EEA95E0DC
:104F60000E944E116DE571E088EA95E00E944E11B5
:104F70006DE571E082EA95E00E944E116DE571E009
:104F80008CE995E00E944E116EED72E086E995E0A5
:104F90000E944E1165EE72E080E995E00E944E118C
:104FA0001092690585E080936A0510926B05109256
:104FB0006D0510926C0510926F0510926E0510929F
:104FC0007005109271056EEE72E083E695E00E9426
:104FD0004E1186E190E090931605809315058CE7BD
:104FE0009CE8A1E0B0E08093210590932205A09376
:104FF0002305B093240581EA97E6A3E3BDEB8093F4
:10500000250590932605A0932705B093280586E6ED
:1050100096E6A6EABFE38093290590932A05A0931C
:105020002B05B0932C0510922D0510922E05109291
:105030002F05109230051092310510923205109212
:1050400033051092340581E08093350529E130E085
:1050500030933705209336058093380580E090E43F
:10506000ACE1B5E48093390590933A05A0933B05F4
:10507000B0933C0510923D0510923E0510923F05FD
:1050800010924005E1E4F5E080E1DF011D928A9590
:10509000E9F71092510510925205109253051092A3
:1050A000540510925505109256051092570510920E
:1050B00058051092590510925A0510925B051092EE
:1050C0005C0510925D0510925E0510925F051092CE
:1050D000600581E090E090936205809361050895FA
:1050E000CF93DF93CDB7DEB72C970FB6F894DEBF22
:1050F0000FBECDBF789484B5826084BD84B58160D5
:1051000084BD85B5826085BD85B5816085BD809192
:105110006E00816080936E0010928100809181000A
:105120008260809381008091810081608093810002
:10513000809180008160809380008091B1008460C4
:105140008093B1008091B00081608093B000809125
:105150007A00846080937A0080917A0082608093E4
:105160007A0080917A00816080937A0080917A0041
:10517000806880937A001092C10061E08EE00E9406
:105180001D03E0917C04F0917D0482E08083E09136
:105190007804F09179041082E0917A04F0917B0414
:1051A0008FEC808310928404E0918004F09181045C
:1051B00086E08083E0917E04F0917F0480818061AD
:1051C0008083E0917E04F0917F04808188608083F9
:1051D000E0917E04F0917F04808180688083E0917B
:1051E0007E04F0917F0480818F7D808360E08EE07B
:1051F0000E94EF020E94FB0781E08093480483E253
:1052000080936A041092490410926B0460E189E073
:1052100095E00E943F0A0E9433088FE39CE90197C2
:10522000F1F700C0000068EC70E080E090E00E94C0
:105230008E0384E690E090930B0180930A010E9414
:1052400095318093E60385E690E00E949531809346
:10525000E7030091E6031091E703B801012E000C6B
:10526000880B990B0E9475309B01AC010E94E433BE
:10527000811106C00B5011090C30110508F4EDC066
:1052800084E690E00E946D1239E6C32E35E0D32EFD
:1052900056010EE110E0C8010E949531F50181939D
:1052A0005F010F5F1F4F07321105A9F710916A05C3
:1052B000612F012E000C770B880B990B0E94753023
:1052C0009B01AC010E94E433811103C0153009F445
:1052D000EFC08EE190E00E94961268EC70E080E0F2
:1052E00090E00E948E036AEF72E08AEB95E00E94E4
:1052F000F8100E94FB0764E670E080E090E00E94F6
:105300008E0366E975E0CE0101960E94451160E0CA
:10531000CE0101960E9490100E948710CE01019646
:105320000E942B106AEB75E0CE0101960E94451198
:10533000CE0101960E94B711CE0101960E942B105A
:1053400086E78093C0058091C9058F3F11F40E94C4
:10535000FB078091C9058F3F01F58091C00591E061
:105360009093480480936A041092490410926B044D
:1053700060ED89E095E00E943F0A0E94330861E0F9
:105380008091C0050E941A091092FB038093FA03D2
:1053900089E095E00E94F809F82EF8E5FF1609F477
:1053A00095C063E073E08AEB95E00E94F8101092DC
:1053B00007016AEB75E0CE0101960E944511CE010E
:1053C00001960E94B711CE0101960E942B108AE22D
:1053D000C82ED12C98EE892E93E0992EA12CB12CB9
:1053E00020E0E22E20E0F22E01E06DE571E0CE013A
:1053F00007960E944E1110E08CE694E00E94F301A3
:10540000181619060CF0D3C01111D1C08CE694E027
:105410000E94D1018A3009F07AC11091E80311236A
:1054200009F48AC18091AC059091AD05892B09F4EE
:105430007CC16FE073E0CE0101960E944E11BE0167
:10544000695F7F4FCE0101960E94C4100E94A9019E
:10545000CE0101960E942B1068C145E1C42E45E0A3
:10546000D42E04E610E0C8010E949531F601819324
:105470006F010F5F1F4F023B1105A9F780911505C2
:1054800090911605909309018093080167E175E0FA
:10549000CE0101960E944E11BE016F5F7F4F86E9DB
:1054A00095E00E94E00FCE0101960E942B10ECCEF9
:1054B0000EE110E0C8010E949531F60181936F0161
:1054C0000F5F1F4F05341105A9F707CF88E80E9429
:1054D000170F9093CE058093CD058AE80E94170F91
:1054E0009093D0058093CF058CE80E94170F90937E
:1054F000D2058093D1058EE80E94170F9093D405B2
:105500008093D30580E90E94170F9093D60580936E
:10551000D50582E90E94170F9093D8058093D7058F
:1055200084E90E94170F9093DA058093D90586E9E4
:105530000E94170F9093DC058093DB0588E90E9499
:10554000170F9093DE058093DD058AE90E94170FFF
:105550009093E0058093DF058CE90E94170F9093EC
:10556000E2058093E1058EE90E94170F9093E40510
:105570008093E3058091C9058F3F09F028CF809182
:10558000C00591E09093480480936A041092490406
:1055900010926B0464EF89E095E00E943F0A6FE38C
:1055A00089E095E00E943F0A0E94330810CF8B8566
:1055B0009C85892B51F08CE694E00E94820264E184
:1055C00070E080E090E00E948E03BE01695F7F4F33
:1055D00088EA95E00E94E00FCE0107960E942B100A
:1055E0006DE571E08AEB95E00E94F8108091AC05C2
:1055F0009091AD058130910509F0C6C068EA75E06B
:1056000084EB95E00E942E110E946B0F64EB75E015
:10561000CE0101960E9445118D819E81892B09F44E
:10562000A5C0E981FA81309709F4A0C08081823455
:1056300009F484C0833409F48EC0813409F096C023
:1056400068E173E088EA95E00E94F810CE010196C7
:105650000E942B1088EA95E00E94BA0FCB010E94AD
:1056600038198091F103882309F43FC00E949D04FA
:10567000A50194010E94F531CA01B9010E9473305D
:105680002091ED033091EE034091EF035091F00330
:105690000E94263220910C0130910D0140910E01A3
:1056A00050910F010E948F331816FCF48091EB0388
:1056B0009091EC034A9609F4A0C08091E90390917F
:1056C000EA030E9438190E949D04A50194010E94DA
:1056D000F531CA01B9010E9473306093ED037093F4
:1056E000EE038093EF039093F0036AE070E080E0B4
:1056F00090E00E948E03E114F10409F476CE0E943A
:10570000FF01882309F471CE0E9400006ECE8D3017
:1057100009F483CE89831A8241E050E0BE016F5FB5
:105720007F4FCE0107960E945B106AE070E080E038
:1057300090E00E948E0360CE11E0F7CF6BE173E042
:1057400088EA95E00E94F8101092F1038CEF9FEF29
:105750000E9438197BCF6EE173E088EA95E00E94E1
:10576000F8100093F1038DEF9FEFF2CFBE016F5F52
:105770007F4F88EA95E00E942E116AE070E080E099
:1057800090E00E948E0362CF049768F56EEC72E0A1
:10579000CE0101960E944E11BE016F5F7F4F88EAD5
:1057A00095E00E94C50F182FCE0101960E942B1084
:1057B0001123C9F08091AC059091AD05029788F056
:1057C000E091A805F091A905309759F081818033C7
:1057D0000CF4845E9601281B310987FD3395C901BD
:1057E0003ECF80E0F6CF8091AC059091AD05029759
:1057F00008F437CF0E94BF1234CF80916905882307
:1058000009F461CF0E947C245ECF83E695E00E947C
:105810002B1080E995E00E942B1086E995E00E940C
:105820002B108CE995E00E942B1082EA95E00E94F3
:105830002B1088EA95E00E942B108EEA95E00E94DA
:105840002B1084EB95E00E942B108AEB95E00E94D0
:105850002B108DE491E09093EF058093EE058EEE92
:1058600095E00C940B07EF920F931F93CF93DF9368
:10587000E80134E047FD34E1042E000C550B57FFDE
:1058800003C0519541955109E32E022F242FAE01FB
:105890000E94B62CCE01DF91CF911F910F91EF9016
:1058A0000895662777270C94152E1F93FC019927DE
:1058B0008827BC01E89411911032E9F3193010F0F7
:1058C0001E30C8F31B3251F01D3249F4689406C0F3
:1058D0000E94872C610F711D811D911D1191105324
:1058E0001A30B0F33EF490958095709561957F4F96
:1058F0008F4F9F4F1F910895BB274A3031F4992352
:1059000022F4BDE2909581959F4F0C949D2C592FC8
:10591000482F372F262F660F771F881F991F660F76
:10592000771F881F991F620F731F841F951F660FB3
:10593000771F881F991F0895BB27FB015527AA27AA
:10594000880F991FAA1FA41710F0A41B839550510C
:10595000B9F7A05DAA3308F0A95DA193009779F784
:10596000B111B1931192CB010C945E30A9E0B0E07B
:10597000ECEBFCE20C94C4316A01F22EB02E102F35
:10598000FBE3AF2EA01608F41BE31F5F012F27E0F7
:10599000AE014F5F5F4F0E94652FBC018981982F38
:1059A0009970913009F43FC09BE2E1FC04C09E2D48
:1059B0009170E0FC3AC05E2D5071E82FE87083FFD3
:1059C00046C084E0911101C083E0EF2DE81B8F15E4
:1059D00008F0E0E0D6018E2F20E2552351F1992303
:1059E00029F0D6019C93C60101966C0196012D5FAA
:1059F0003F4FE2FE24C08EE4D6018C9391E41196D1
:105A00009C93119712968C93D9018E2F90E281115D
:105A10001BC0E20FF32FF11D10828EEF9FEF29962E
:105A2000ECE00C94E0319DE2C6CF90E2C4CF2D9320
:105A300081508111FCCFCE0ED11CE0E0D0CF8EE69C
:105A4000D6018C9391E6DBCF9D938150E0CF482F18
:105A5000447082FF3DC084E0911101C083E08F1546
:105A600010F4EF2DE81BD6018E2F20E2552309F10B
:105A7000992329F0D6019C93C60101966C019601E9
:105A80002D5F3F4FE2FE1BC089E4D6018C938EE46C
:105A900011968C93119786E412968C93D9018E2FD0
:105AA00090E2882309F4B5CF9D938150FACF2D93CE
:105AB00081508111FCCFCE0ED11CE0E0D9CF89E618
:105AC000D6018C938EE611968C93119786E6E4CFDF
:105AD0009B0177FF02C030E020E0A1E0B0E091112F
:105AE00002C0B0E0A0E0F9013196AE0FBF1F8B2CD1
:105AF000912CBB2009F461C05401EFEFAE1ABE0A2D
:105B0000AA0DBB1DFA161B0619F014F04F2D4A1BE7
:105B1000511188C0E3FC59C07601A42FB0E2A11155
:105B20004FC0C40ED11C992309F45BC040E0D601DC
:105B30001196F60190836D01552309F448C0012F99
:105B4000060F9A81582F507184FF03C0913309F4D6
:105B5000015010160CF047C0093008F008E0EEE2E2
:105B6000FE2E5B01A01AB1088501919481949108E1
:105B70002F3F320729F4D601FC92F60131966F01CE
:105B80006217730794F1021713077CF5DB01A21B60
:105B9000B30BAA24A394B12CAC0EBD1EAA0DBB1D41
:105BA00011968C9121503109D6011196281539058D
:105BB000F4F0F60180836D01DBCFB12CA12CA0CFD6
:105BC000F701B1937F01A150AACF9111B0CFD601B7
:105BD000942F50E302C05D9391509111FCCFC40EFD
:105BE000D11C40E0ACCF01E0BACF80E3DBCF62173D
:105BF000730731F4963388F4953311F4552369F023
:105C0000F6018083FD01842F90E2811108C0A40F6A
:105C1000B11D1C9290E080E002CF81E3F1CF91931F
:105C20008150F3CF911183CF8ACFB0E0A0E0EBE1B8
:105C3000FEE20C94C4315C017B016115710519F021
:105C4000DB018D939C9385010F5F1F4FF501D08180
:105C50008D2F90E00E943D306C01892BB9F5DD322B
:105C6000B9F50F5F1F4FD5011196DC91C1E05801C6
:105C7000F1E0AF1AB10843E050E062EF70E0C50117
:105C80000E944630892B69F5680182E0C80ED11C5C
:105C900045E050E06DEE70E0C6010E944630892B71
:105CA00021F4680197E0C90ED11CE114F10419F048
:105CB000D701CD92DC9260E070E080E89FEFC111E7
:105CC000FFC060E070E080E89FE7FAC05801BBCFFA
:105CD000DB3229F485010E5F1F4FF501D181C0E051
:105CE000C6CF43E050E06AEE70E0C5010E94463046
:105CF000892BE9F0F80110E000E020E030E0A90194
:105D00005F01B0ED8B2E8D0E89E08815C8F19C2EB9
:105D1000689491F88C2F8870C2FF16C0811102C060
:105D20000F5F1F4F3196D501DC91C92DE9CFE114EA
:105D3000F10429F00E5F1F4FF7011183008360E02B
:105D400070E080EC9FE7BCC0882311F0015011097E
:105D5000A5E0B0E00E94AB319B01AC01220F331FE4
:105D6000441F551F280D311D411D511D283999E92A
:105D70003907490799E15907A8F2C6609C2ED2CF8E
:105D8000AEEF8A1206C0C3FD3CC09C2E689493F807
:105D9000C9CFDF7DD534A9F580818D3239F4C0615A
:105DA000DF011296818162E070E006C0DF018B3274
:105DB000C1F3119661E070E080535D01A61AB70A45
:105DC0008A30F8F4E0E8CE16ECE0DE065CF4B601CA
:105DD000660F771F660F771FC60ED71ECC0CDD1C13
:105DE000C80ED11C5D01FFEFAF1ABF0A8C91805322
:105DF0008A30A8F1C4FF03C0D194C194D1080C0D1E
:105E00001D1DC1FF09C0E114F10431F081E0A81AA1
:105E1000B108D701AD92BC92CA01B9010E9473309A
:105E2000C370C33009F490584B015C0120E030E0AE
:105E3000A9010E946E30882309F440C0C1E2D1E07C
:105E400017FF05C0119501951109C9E0D1E06E0158
:105E5000B8E1CB1AD10880E2E82EF12C0FC0D501B1
:105E6000B1CFFE0125913591459154910E191F092D
:105E7000C501B4010E94D4304B015C01D501C401BD
:105E80000E151F0574F72497F594E794CC16DD06DC
:105E9000A9F78A2F880F8B2F881F8F3F49F020E0AA
:105EA00030E0A901C501B4010E946E30811106C025
:105EB00082E290E090931C0680931B06C501B4011A
:105EC000CDB7DEB7ECE00C94E031283008F027E0E5
:105ED0003327DA01990F311D87FD91600096610526
:105EE000710539F432602E5F3D9330E32A95E1F776
:105EF00008959F3F30F080387105610509F03C5FDF
:105F00003C5F3D93913008F08068911DDF93CF9303
:105F10001F930F93FF92EF92192F987F9695E92F79
:105F200096959695E90FFF27E158FE4F992733275D
:105F3000EE24FF24A701E70105900894079428F4B4
:105F4000360FE71EF81E491F511D660F771F881F69
:105F5000991F0694A1F70590079428F4E70EF81E00
:105F6000491F561FC11D770F881F991F661F069472
:105F7000A1F70590079428F4F80E491F561FC71F74
:105F8000D11D880F991F661F771F0694A1F70590F2
:105F9000079420F4490F561FC71FD81F990F661F7B
:105FA000771F881F0694A9F784911095177041F008
:105FB000D695C79557954795F794E7941A95C1F7E5
:105FC000E5E2F1E068941590159135916591959110
:105FD00005907FE27395E118F10A430B560BC90B4C
:105FE000D009C0F7E10CF11E431F561FC91FD01D79
:105FF0007EF4703311F48A95E6CFE894015030F0C6
:10600000080F0AF40027021708F4202F2395022F07
:106010007A3328F079E37D932A95E9F710C07D93D0
:106020002A9589F60694979567953795179517944D
:10603000E118F10A430B560BC90BD00998F02395D0
:106040007E9173957A3308F070E37C932013B8F750
:106050007E9170617D9330F0839571E37D9370E361
:106060002A95E1F71124EF90FF900F911F91CF91A6
:10607000DF91992787FD9095089591110C944131F6
:10608000803219F089508550C8F70895FB01DC0172
:106090004150504088F08D9181341CF08B350CF4C8
:1060A000805E659161341CF06B350CF4605E861B7C
:1060B000611171F3990B0895881BFCCFDC01FC0181
:1060C000672F71917723E1F7329704C07C916D932C
:1060D00070836291AE17BF07C8F308950E94B03075
:1060E00008F481E00895E89409C097FB3EF4909588
:1060F0008095709561957F4F8F4F9F4F9923A9F0A1
:10610000F92F96E9BB279395F6958795779567952F
:10611000B795F111F8CFFAF4BB0F11F460FF1BC073
:106120006F5F7F4F8F4F9F4F16C0882311F096E906
:1061300011C0772321F09EE8872F762F05C06623B4
:1061400071F096E8862F70E060E02AF09A95660F6D
:10615000771F881FDAF7880F9695879597F9089526
:10616000990F0008550FAA0BE0E8FEEF1616170668
:10617000E807F907C0F012161306E407F50798F0D0
:10618000621B730B840B950B39F40A2661F0232BE9
:10619000242B252B21F408950A2609F4A140A69565
:1061A0008FEF811D811D08950E94E7300C945B31B3
:1061B0000E944D3138F00E94543120F0952311F0A7
:1061C0000C9444310C944A3111240C948F310E9468
:1061D0006C3170F3959FC1F3950F50E0551F629F8E
:1061E000F001729FBB27F00DB11D639FAA27F00D30
:1061F000B11DAA1F649F6627B00DA11D661F829F57
:106200002227B00DA11D621F739FB00DA11D621F3B
:10621000839FA00D611D221F749F3327A00D611D58
:10622000231F849F600D211D822F762F6A2F11243A
:106230009F5750409AF0F1F088234AF0EE0FFF1F6D
:10624000BB1F661F771F881F91505040A9F79E3FC4
:10625000510580F00C9444310C948F315F3FE4F38E
:10626000983ED4F3869577956795B795F795E7951A
:106270009F5FC1F7FE2B880F911D9695879597F923
:10628000089599278827089597F99F6780E870E017
:1062900060E008959FEF80EC089500240A9416169C
:1062A000170618060906089500240A941216130604
:1062B000140605060895092E0394000C11F4882392
:1062C00052F0BB0F40F4BF2B11F460FF04C06F5FAE
:1062D0007F4F8F4F9F4F089557FD9058440F551F84
:1062E00059F05F3F71F04795880F97FB991F61F058
:1062F0009F3F79F087950895121613061406551FCF
:10630000F2CF4695F1DF08C0161617061806991F3A
:10631000F1CF86957105610508940895E894BB272F
:1063200066277727CB0197F90895F999FECF92BD9B
:1063300081BDF89A992780B50895262FF999FECF47
:106340001FBA92BD81BD20BD0FB6F894FA9AF99A92
:106350000FBE019608950E941732A59F900DB49F1D
:10636000900DA49F800D911D11240895B7FF0C94EA
:10637000AB310E94AB31821B930B08952F923F9259
:106380004F925F926F927F928F929F92AF92BF9245
:10639000CF92DF92EF92FF920F931F93CF93DF93F1
:1063A000CDB7DEB7CA1BDB0B0FB6F894DEBF0FBE4E
:1063B000CDBF09942A88398848885F846E847D849B
:1063C0008C849B84AA84B984C884DF80EE80FD809D
:1063D0000C811B81AA81B981CE0FD11D0FB6F89413
:1063E000DEBF0FBECDBFED010895A1E21A2EAA1B9C
:1063F000BB1BFD010DC0AA1FBB1FEE1FFF1FA21775
:10640000B307E407F50720F0A21BB30BE40BF50B71
:10641000661F771F881F991F1A9469F760957095FA
:10642000809590959B01AC01BD01CF010895A29F7D
:10643000B001B39FC001A39F700D811D1124911D58
:10644000B29F700D811D1124911D08955058BB27D6
:10645000AA270E943E320C945B310E944D3138F0E5
:106460000E94543120F039F49F3F19F426F40C9423
:106470004A310EF4E095E7FB0C944431E92F0E9479
:106480006C3158F3BA17620773078407950720F039
:1064900079F4A6F50C948E310EF4E0950B2EBA2FFC
:1064A000A02D0B01B90190010C01CA01A00111241A
:1064B000FF27591B99F0593F50F4503E68F11A16C6
:1064C000F040A22F232F342F4427585FF3CF469557
:1064D00037952795A795F0405395C9F77EF41F1679
:1064E000BA0B620B730B840BBAF09150A1F0FF0F43
:1064F000BB1F661F771F881FC2F70EC0BA0F621F2F
:10650000731F841F48F4879577956795B795F7951E
:106510009E3F08F0B0CF9395880F08F09927EE0FB3
:106520009795879508950E94A7320C945B310E943D
:10653000543158F00E944D3140F029F45F3F29F06A
:106540000C94443151110C948F310C944A310E94B7
:106550006C3168F39923B1F3552391F3951B550BD7
:10656000BB27AA2762177307840738F09F5F5F4F26
:10657000220F331F441FAA1FA9F335D00E2E3AF065
:10658000E0E832D091505040E695001CCAF72BD07D
:10659000FE2F29D0660F771F881FBB1F26173707CE
:1065A0004807AB07B0E809F0BB0B802DBF01FF2700
:1065B00093585F4F3AF09E3F510578F00C94443168
:1065C0000C948F315F3FE4F3983ED4F38695779532
:1065D0006795B795F7959F5FC9F7880F911D9695B9
:1065E000879597F90895E1E0660F771F881FBB1F15
:1065F000621773078407BA0720F0621B730B840BC2
:10660000BA0BEE1F88F7E09508950E940C3368944A
:10661000B1110C948F3108950E94743188F09F5706
:1066200098F0B92F9927B751B0F0E1F0660F771FB6
:10663000881F991F1AF0BA95C9F714C0B13091F0AC
:106640000E948E31B1E008950C948E31672F782F1F
:106650008827B85F39F0B93FCCF386957795679571
:10666000B395D9F73EF490958095709561957F4FDD
:106670008F4F9F4F089597FB16F40E947F330C9421
:106680004233E894F92F96EBFF2381F0121613069C
:106690001406440B9395F6958795779567955795CE
:1066A0004040FF23B9F71BC099270895882351F470
:1066B0009850D2F7872B762F652F542F432F322FE8
:1066C00020E0B1F3121613061406440B88233AF0A7
:1066D0009A95440F551F661F771F881FCAF75523C9
:1066E0004AF4440F551F11F460FF04C06F5F7F4FE1
:1066F0008F4F9F4F880F9695879597F9089590959E
:1067000080957095609550954095309521953F4FB7
:106710004F4F5F4F6F4F7F4F8F4F9F4F08950E9496
:10672000B03008F48FEF0895FA01EE0FFF1F309696
:1067300021053105A1F16115710561F48038BFE3D0
:106740009B0749F168949038810561F08038BFEF6C
:106750009B0741F099234AF5FF3FE10531052105EB
:1067600019F1E8940894E795D901AA2329F4AB2FED
:10677000BE2FF85FD0F310C0FF5F70F4A695E0F76E
:10678000F73950F019F0FF3A38F49F779F930DD006
:106790000F9007FC9058089546F00C944A3160E041
:1067A00070E080E89FE308954FE79F775F934F93F2
:1067B0003F932F930E9494342F913F914F915F917B
:1067C0000E94D4300C94F1330E94B030880B990BA6
:1067D000089529F416F00C9444310C948E310C94E5
:1067E0004A310E947431A8F39638A0F707F80F9247
:1067F000E8942BE33AEA48EB5FE70E94EA300F9215
:106800000F920F924DB75EB70F920E94DC34E8E60C
:10681000F0E00E9423344F915F91EF91FF91E59555
:10682000EE1FFF1F49F0FE57E0684427EE0F441F9C
:10683000FA95E1F74195550B0E9456340F9007FEEB
:106840000C944A340895DF93CF931F930F93FF92D4
:10685000EF92DF927B018C01689406C0DA2EEF0183
:106860000E94E730FE01E894A5912591359145916C
:106870005591A6F3EF010E943E32FE019701A80157
:10688000DA9469F7DF90EF90FF900F911F91CF910D
:10689000DF9108959B01AC0160E070E080E89FE328
:1068A0000C9493320C9444310C9410350E94743142
:1068B000D8F39923C9F3940F511DA3F3915050407D
:1068C00094F059F0882332F0660F771F881F91509B
:1068D0005040C1F79E3F51052CF7880F911D9695AA
:1068E000879597F908955F3FACF0983E9CF0BB27E1
:1068F000869577956795B79508F4B1609395C1F73C
:10690000BB0F58F711F460FFE8CF6F5F7F4F8F4FD9
:106910009F4FE3CF0C948F3116F00C9410350C94EC
:106920004A3168940C9444310E947431A8F399233D
:10693000C1F3AEF3DF93CF931F930F93FF92C92F51
:10694000DD2788232AF02197660F771F881FDAF743
:1069500020E030E040E85FEB9FE3883920F0803EA4
:1069600038F021968F770E942732E0E9F0E004C0EA
:106970000E942732EDEBF0E00E9423348B01BE0130
:10698000EC01FB2E6F5771097595771F880B990BDA
:106990000E94753028E132E741E35FE30E94E7306F
:1069A000AF2D9801AE01FF900F911F91CF91DF9114
:1069B0000E943E320C945B31FA01DC01AA0FBB1F2E
:1069C0009B01AC01BF5728F4222733274427507876
:1069D00020C0B75190F4AB2F0024469537952795EA
:1069E000011CA395D2F3002071F0220F331F441F26
:1069F000B395DAF30ED00C94263261307105A0E81D
:106A00008A07B94630F49B01AC01662777278827AF
:106A10009078309621F02083318342835383089508
:106A20009F3F31F0915020F4879577956795B79502
:106A3000880F911D9695879597F90895DB018F939F
:106A40009F930E94AB31BF91AF91A29F800D911D8A
:106A5000A39F900DB29F900D11240895AA1BBB1BFC
:106A600051E107C0AA1FBB1FA617B70710F0A61B4E
:106A7000B70B881F991F5A95A9F780959095BC016F
:106A8000CD01089597FB072E16F4009407D077FDEB
:106A900009D00E942E3507FC05D03EF490958195D3
:106AA0009F4F0895709561957F4F0895EE0FFF1FDA
:106AB0000590F491E02D0994DF93CF931F930F93EA
:106AC0009A9DF02D219FF00D8B9DF00D8A9DE02D5C
:106AD000F10D039FF00D029FE00DF11D4E9DE00DA5
:106AE000F11D5E9DF00D4F9DF00D7F936F93BF9252
:106AF000AF925F934F93D5010E9417328B01AC0187
:106B0000D7010E941732EB01E80FF91FD6010E944E
:106B1000AB352F913F91D6010E941732C60FD71F78
:106B2000E81FF91FAF91BF910E94AB352F913F91A4
:106B30000E941732C60FD71FE81FF91FD6010E9407
:106B40001732E60FF71F9801BE01CF010F911F9179
:106B5000CF91DF9108950E941732460F571FC81F2B
:106B6000D91F08F431960895689401C0E894F92F6C
:106B7000F12B12F00C94E835A0E0B0E0E2ECF5E384
:106B80000C94C431092E059422F40E94443611233A
:106B900092F4F0E80F26FFEFE094F0940095109542
:106BA000B094C094D094A194BF0ACF0ADF0AEF0A30
:106BB000FF0A0F0B1F0B0E94F33507FC0E9444369F
:106BC000CDB7DEB7ECE00C94E031689401C0E894F6
:106BD0008F929F92CF93DF930E94F335DF91CF91F5
:106BE0009F908F90089588249924F401E401B0E4E3
:106BF0009F93AA279A158B049C04ED05FE05CF05EB
:106C0000D007A10798F4AD2FDC2FCF2FFE2FE92D51
:106C1000982C892E982F872F762F652F542F432F4E
:106C2000322F2227B85031F7BF9127C01B2EBF91BA
:106C3000BB27220F331F441F551F661F771F881F56
:106C4000991F881C991CEE1FFF1FCC1FDD1FAA1F58
:106C5000BB1F8A149B04EC05FD05CE05DF05A007CC
:106C6000B10748F08A189B08EC09FD09CE09DF0935
:106C7000A00BB10B21601A94E1F62EF49401AF0140
:106C8000BE01CD01000C089560957095809590959A
:106C900030954095509521953F4F4F4F5F4F6F4F27
:106CA0007F4F8F4F9F4F0895002E083090F0982F00
:106CB000872F762F652F542F432F322F22270850EE
:106CC000F4CF220F331F441F551F661F771F881FE5
:106CD000991F0A95B2F7002D089597FD1094002E84
:106CE000083098F00850232F342F452F562F672F48
:106CF000782F892F912DF4CF1594979587957795B7
:106D0000679557954795379527950A95AAF71124C2
:106D1000002D08952A0D3B1D4C1D5D1D6E1D7F1D10
:106D2000801F911F08952A193B094C095D096E09BE
:106D30007F09800B910B08950024A7FD00942A176A
:106D400030054005500560057005800590050895E3
:106D50000F931F93CF93DF938230910510F482E05D
:106D600090E0E0911F06F091200630E020E0B0E0D6
:106D7000A0E0309799F42115310509F44AC0281B89
:106D8000390B24303105D8F58A819B816115710555
:106D900089F1FB0193838283FE0111C040815181FF
:106DA0000281138148175907E0F04817590799F4F1
:106DB000109761F012960C93129713961C933296CB
:106DC000CF01DF91CF911F910F91089500931F067E
:106DD00010932006F4CF2115310551F042175307C7
:106DE00038F0A901DB019A01BD01DF01F801C1CF33
:106DF000EF01F9CF9093200680931F06CDCFFE01BF
:106E0000E20FF31F81939193225031093983288334
:106E1000D7CF20911D0630911E06232B41F42091DF
:106E200012013091130130931E0620931D0620910C
:106E30001001309111012115310541F42DB73EB7F4
:106E40004091140150911501241B350BE0911D0652
:106E5000F0911E06E217F307A0F42E1B3F0B281734
:106E6000390778F0AC014E5F5F4F2417350748F0C3
:106E70004E0F5F1F50931E0640931D068193919302
:106E80009FCFF0E0E0E09CCFCF93DF930097E9F055
:106E9000FC01329713821282A0911F06B091200646
:106EA000ED0130E020E01097A1F420813181820FC4
:106EB000931F20911D0630911E062817390709F0EF
:106EC00061C0F0931E06E0931D06DF91CF910895F7
:106ED000EA01CE17DF07E8F54A815B819E01411583
:106EE0005105B1F7E901FB83EA8349915991C40F38
:106EF000D51FEC17FD0761F4808191810296840F04
:106F0000951FE90199838883828193819B838A837A
:106F1000F0E0E0E012968D919C9113970097B9F5FF
:106F20002D913C911197CD010296820F931F2091D4
:106F30001D0630911E062817390739F6309751F58E
:106F40001092200610921F06B0931E06A0931D06F5
:106F5000BCCFD383C28340815181840F951FC81752
:106F6000D90761F44E5F5F4F88819981480F591F9F
:106F7000518340838A819B819383828321153105CC
:106F800009F0B0CFF0932006E0931F069ECFFD01DD
:106F9000DC01C0CF13821282D7CFB0E0A0E0E3EDD6
:106FA000F7E30C94C0318C01009751F4CB010E949F
:106FB000A8368C01C801CDB7DEB7E0E10C94DC3116
:106FC000FC01E60FF71F9C0122503109E217F3077D
:106FD00008F49DC0D901CD91DC911197C617D70750
:106FE00098F0C530D10530F3CE0104978617970786
:106FF00008F3C61BD70B2297C193D1936D937C9353
:10700000CF010E944437D6CF5B01AC1ABD0A4C01B8
:107010008C0E9D1EA0911F06B0912006512C412C74
:10702000F12CE12C109731F580911D0690911E06F0
:107030008815990509F05CC04616570608F058C037
:107040008091100190911101009741F48DB79EB786
:107050004091140150911501841B950BE817F90715
:1070600008F055C0F0931E06E0931D06F9017183E8
:107070006083A0CF8D919C91119712966C9012977E
:1070800013967C901397A815B90559F56C0142E049
:10709000C40ED11CCA14DB0420F1AC014A195B09EF
:1070A000DA011296159780F06282738251834083D1
:1070B000D9016D937C93E114F10471F0D70113961B
:1070C000FC93EE93129776CF22968C0F9D1FF901B9
:1070D00091838083F301EFCFF0932006E0931F06A6
:1070E00069CF4816590608F42C017D01D3019ACFC7
:1070F000CB010E94A8367C01009749F0AE01B8018F
:107100000E949238C8010E944437870153CF10E093
:1071100000E050CF9111089581568A5108F48052B1
:1071200085580895FB01DC0102C001900D92415089
:107130005040D8F70895FB01DC0101900D9200202A
:10714000E1F70895FB01DC014150504030F08D9192
:107150000190801919F40020B9F7881B990B089544
:10716000FB01DC014150504048F001900D9200209D
:10717000C9F701C01D9241505040E0F70895FB014E
:1071800051915523A9F0BF01DC014D9145174111E3
:10719000E1F759F4CD010190002049F04D914015DF
:1071A0004111C9F3FB014111EFCF81E090E001975C
:1071B000089511E0CEE4D1E004C0FE010E945635EE
:1071C0002196CF34D107C9F7F894FFCF0000A04033
:1071D000C8000101160064000000F0410000210613
:1071E00080005E00BC007701FF0186000000000007
:1071F000790000000035027C01C2018202F301D156
:1072000001E501000000003F0A120A6E0A43060B66
:107210000AF809E9090000000044067C016E0A43EF
:1072200006A006B8062B060D0A0052454200564538
:1072300052002356657273696F6E3A004C4F4700D7
:10724000234C6F67676572204E616D653A00534845
:107250004F57533D00474554007320005341564556
:107260003D0054494D45493D0023496E7465727691
:10727000616C3D0054494D45443D002344757261A5
:1072800074696F6E3D004448543D0042543D0053C4
:107290004C20503D00506120756E6C696B656C79B7
:1072A0002100685061004E45543D0055565A002358
:1072B00055562056303D005620004D533D002C00C1
:1072C00023496E636F727265637421204D533D31A3
:1072D000323344334435005428312C322C33293D89
:1072E00000206F4320445320546865726D6F6D65B4
:1072F0007465720020572F6D5E3200555620496E1E
:1073000074656E7369747900572F6D5E3220005575
:10731000563D0070706D00434F323D00206E672F68
:107320004C00504D28312E302C322E352C31302946
:107330003D006F432000483D00250068506120005B
:107340006F430020413D004C6967687420496E74AA
:10735000656E7369747900206C7820004C3D00499B
:107360005220466C616D65204C6576656C3D00472A
:107370006173206C6576656C3D00204D756C746999
:1073800073656E736F72730023456E61626C650086
:107390002344697361626C650044440023496E763E
:1073A000616C6964206B65792100424E4D4C30332D
:1073B000006E616E6F4232693600234E6F20536556
:1073C0006E736F72210057656C636F6D653A0023B1
:1073D000626D70206661696C6564007365726961D5
:0E73E0006C3A20002D35002D34002D330000B6
:107E0000112484B714BE81FFF0D085E080938100F7
:107E100082E08093C00088E18093C10086E0809377
:107E2000C20080E18093C4008EE0C9D0259A86E02C
:107E300020E33CEF91E0309385002093840096BBD3
:107E4000B09BFECF1D9AA8958150A9F7CC24DD24C4
:107E500088248394B5E0AB2EA1E19A2EF3E0BF2EE7
:107E6000A2D0813461F49FD0082FAFD0023811F036
:107E7000013811F484E001C083E08DD089C08234E0
:107E800011F484E103C0853419F485E0A6D080C0E4
:107E9000853579F488D0E82EFF2485D0082F10E0AE
:107EA000102F00270E291F29000F111F8ED06801E7
:107EB0006FC0863521F484E090D080E0DECF843638
:107EC00009F040C070D06FD0082F6DD080E0C81688
:107ED00080E7D80618F4F601B7BEE895C0E0D1E017
:107EE00062D089930C17E1F7F0E0CF16F0E7DF06D8
:107EF00018F0F601B7BEE89568D007B600FCFDCFD4
:107F0000A601A0E0B1E02C9130E011968C91119780
:107F100090E0982F8827822B932B1296FA010C0160
:107F200087BEE89511244E5F5F4FF1E0A038BF0790
:107F300051F7F601A7BEE89507B600FCFDCF97BE46
:107F4000E89526C08437B1F42ED02DD0F82E2BD052
:107F50003CD0F601EF2C8F010F5F1F4F84911BD097
:107F6000EA94F801C1F70894C11CD11CFA94CF0C13
:107F7000D11C0EC0853739F428D08EE10CD085E9AC
:107F80000AD08FE07ACF813511F488E018D01DD067
:107F900080E101D065CF982F8091C00085FFFCCF94
:107FA0009093C60008958091C00087FFFCCF809118
:107FB000C00084FD01C0A8958091C6000895E0E648
:107FC000F0E098E1908380830895EDDF803219F02E
:107FD00088E0F5DFFFCF84E1DECF1F93182FE3DFCA
:107FE0001150E9F7F2DF1F91089580E0E8DFEE27F6
:047FF000FF270994CA
:027FFE00040479
:00000001FF
